:020000040801F1
:10C00000C0CB002051C30108D9F7010871F2010823
:10C0100021F6010825E10108990702080000000047
:10C02000000000000000000000000000B9C201088C
:10C0300073E9010800000000FDC2010831FE01089B
:10C040006BC3010869F801086BC3010845FB0108CF
:10C050006BC301086BC30108A5ED010815EE0108CB
:10C0600037EE010857EE010879EE010869E1010891
:10C07000DDE1010851E20108D1E2010851E30108C4
:10C08000D1E3010851E401086BC301086BC3010847
:10C090006BC301086BC301086BC3010899EE01086B
:10C0A0006BC301086BC301086BC301086BC30108B4
:10C0B00019FF01083DFF010865FF01086BC3010876
:10C0C0006BC301086BC301086BC301086BC3010894
:10C0D0006BC301080904020885040208010502086F
:10C0E000C5ED0108E9FA01086BC301086BC301083B
:10C0F0006BC301086BC301086BC301086BC3010864
:10C100006BC301086BC301088DFF01086BC30108F5
:10C1100069000208E9000208B5FF0108DDFF010817
:10C12000D1E4010851E50108D1E5010855E601080F
:10C1300000F002F800F0B0F80AA090E8000C824489
:10C140008344AAF10107DA4501D100F0A5F8AFF266
:10C15000090EBAE80F0013F0010F18BFFB1A43F0E5
:10C1600001031847A4790000C47900000A444FF085
:10C17000000C10F8013B13F0070408BF10F8014B46
:10C180001D1108BF10F8015B641E05D010F8016B8B
:10C19000641E01F8016BF9D113F0080F1EBF10F8EF
:10C1A000014BAD1C0C1B09D16D1E58BF01F801CB12
:10C1B000FAD505E014F8016B01F8016B6D1EF9D595
:10C1C0009142D6D3704700000023002400250026AA
:10C1D000103A28BF78C1FBD8520728BF30C148BFEA
:10C1E0000B6070476E2900F0B581702900F09B82CA
:10C1F000662907F08F82652907F08C82672907F08E
:10C200008982612907F0888203681B0A28BF41F0F0
:10C210008001692900F06281642900F05F8175293D
:10C2200000F05C816F2900F02882782900F0678295
:10C23000E92900F07387E42900F07087F52900F000
:10C240006D87EF2900F02582F82900F066820368E7
:10C25000DB0928BF41F08001632900F02A87732998
:10C2600000F02F87E32900F04D87F32900F0528773
:10C27000002070471FB500F0EBFF040000200021F4
:10C2800006F07EFD401C60600020002106F08EFD5F
:10C29000E0601FBD10B510BD01F0A8FA1146FFF710
:10C2A000E9FF04F065FE01F0D4FA03B4FFF7F2FFF2
:10C2B00003BC04F073FC0000224B19680868B0E866
:10C2C000F00F80F30988BFF36F8F4FF0000080F309
:10C2D00011884EF00D0E70470000000006480068FF
:10C2E000006880F3088862B661B6BFF34F8FBFF372
:10C2F0006F8F00DF00BF00BF08ED00E0EFF30980A3
:10C30000BFF36F8F0F4B1A6820E9F00F106008B56C
:10C310004FF0500080F31188BFF34F8FBFF36F8F42
:10C3200005F060FF4FF0000080F31188BDE8084081
:10C3300019680868B0E8F00F80F30988BFF36F8FC1
:10C34000704700BF48010020EFF3058070470000F0
:10C350000948804709480047FEE7FEE7FEE7FEE799
:10C36000FEE7FEE7FEE7FEE7FEE7FEE704480549D5
:10C37000054A064B70470000A9FE010831C10108BB
:10C38000C09B0020C0CB0020C0AB0020C0AB002071
:10C39000704700007CB51D4616460C00009001D089
:10C3A0002044401E074B7B442A4669460190304694
:10C3B00000F055FE05461CB10020694600F062FE03
:10C3C00028467CBDE50C00000FB4044910B503AA53
:10C3D000029800F07BFE10BC5DF814FB9800002072
:10C3E0000FB47CB50C0009AA009001D02044401E77
:10C3F000084B7B4469460190089800F030FE0546E2
:10C400001CB10020694600F03DFE28467CBC5DF86A
:10C4100014FB0000990C000070B5044685690068A3
:10C42000C10601D5302600E02026C00707D070BD28
:10C43000D4E9012130469047206A401C20626D1EDD
:10C44000F6D570BD70B5044685690078C00707D180
:10C4500070BDD4E9012120209047206A401C206251
:10C460006D1EF6D570BD09684A0501D540B270470A
:10C47000C905FCD500B2704709684A0501D5C0B2AC
:10C480007047C905FCD580B2704770B50C460546AB
:10C49000012A05D02878800600D5EA69002302E049
:10C4A000012305E05B1C934202D2E05C0028F9D135
:10C4B000A869E618C01AA861286A184428622846A4
:10C4C000FFF7AAFF04E0D5E9012114F8010B90471A
:10C4D000B442F8D32846FFF7B5FF70BD2DE9F0410F
:10C4E0000646002410687529314616A510D0FFF7BE
:10C4F000BAFF002802DA404213A507E031688A0734
:10C5000001D512A502E0490704D511A5012401E0D7
:10C51000FFF7B2FF00210A2206F1240709E0B0FB71
:10C52000F2FCB0FBF2F302FB1C00303078541846EA
:10C53000491C0028F3D123462A463046BDE8F04185
:10C5400000F01FBB000000002D0000002B000000C9
:10C550002000000011680268006A530501D50870C8
:10C560000AE0D30501D5088006E0130603D5C217FB
:10C57000C1E9000200E00860012070472DE9FF5F7B
:10C5800015468A460446DFF8AC80F8440027D8E90F
:10C5900000103E46CDE9001010E03AF816106A4649
:10C5A00002A800F031FE411C07D02178890603D58E
:10C5B000E269391891420DD80744761C207880062C
:10C5C00002D5E069B84205DDAE42E6DB3AF8160076
:10C5D0000028E2D1A069C01BA0612046FFF71CFF24
:10C5E000D8E90010CDE90010002017E03AF8181043
:10C5F0006A4602A800F008FEB0F1FF3F81460BD06A
:10C6000000250DF1080B05E0D4E901211BF8050018
:10C6100090476D1C4D45F7D308F10100B0428046AC
:10C62000E4DB206A384420622046FFF70BFFBDE8B8
:10C63000FF9F0000A673000030B4002100F1240425
:10C6400008E002F00705D208303542EA4372DB0801
:10C650006554491C52EA0305F3D10468002310A273
:10C66000250707D5A40600D421B1C46901230DA272
:10C67000641EC46130BC00F084BA10B50446214683
:10C680001068FFF7F9FE02462046BDE8104000237F
:10C69000D2E7D21D22F00701D1E90023CCE7000048
:10C6A0000000000030000000F0B40D4601880905CC
:10C6B00002D5214C7C4402E01F4C7C440E34002106
:10C6C00000F1240608E002F00F071209E75D42EAD4
:10C6D00003721B097754491C52EA0307F3D102780D
:10C6E0000023120704D5702D06D009B1022311349E
:10C6F0002246F0BC00F045BA01231034F8E770B5CB
:10C7000004460D4621461068FFF7B6FE024629464C
:10C710002046BDE870400023C6E7D21D22F0070383
:10C72000D3E90023C0E70368126843F020030360E5
:10C730000823C3610023B7E7847200002DE9F05F8E
:10C74000894604464FF0000ADFF874B1FB44C0F894
:10C7500020A02046E1688847002874D0252806D00C
:10C76000D4E901219047206A401C2062F1E70026AD
:10C770005F462046E16888472028054607DB312DC3
:10C7800005D2781910F8200C08B10643F1E7B0077C
:10C7900001D526F00406C4F81CA00027C4F818A090
:10C7A0002A2D09D0284604F0F2F938B304EB8708A3
:10C7B000303DC8F8185019E059F8041B204604EB26
:10C7C00087029161E1688847012F054618D1E06929
:10C7D000002820DA26F020061DE0D8F8180000EB2B
:10C7E000800005EB40003038C8F818002046E168AA
:10C7F0008847054604F0CBF90028EED1012F0AD076
:10C800002E2D08D12046E16888477F1C0546022F5F
:10C8100046F02006C4DBA069002803DA404246F057
:10C820000106A061F00701D026F010066C2D0BD098
:10C83000682D09D04C2D39D06A2D35D0742D35D0C6
:10C840007A2D33D016E038E0E1682F46204688473D
:10C85000B842054609D16C2F26D04FF48060E168BC
:10C86000064320468847054604E06C2F1AD04FF453
:10C87000807006430DB3A5F14100192802D8203578
:10C8800046F400664A462946204626604E46FFF793
:10C89000A9FC80B101280BD0F61D26F0070000F19D
:10C8A000080956E74020E4E78020D8E70020D6E7D3
:10C8B00006F104094DE7284652E7206ABDE8F09FDB
:10C8C0001472000070B5064600F04CF90468054685
:10C8D00030460A22002100F05FFC2C6070BD40EA67
:10C8E0000103024630B59B0710D14FF0013400E040
:10C8F00008C208C91D1B9D4315EAC41FF8D013F0D8
:10C90000FF0102F8011B0DD01B0AF8E711F8013BEB
:10C91000002B02F8013B05D011F8013B002B02F877
:10C92000013BF3D130BD10B5431C02E010F8011BF0
:10C9300071B18107FAD14FF0013202C88C1A8C43D1
:10C9400014EAC211F9D0C01A0A0603D0C01E10BDE5
:10C95000C01A10BD0A0401D0801E10BD0902FCD00F
:10C96000401E10BD032A40F2308010F0030C00F08E
:10C97000158011F8013BBCF1020F624498BF11F819
:10C9800001CB00F8013B38BF11F8013BA2F10402D2
:10C9900098BF00F801CB38BF00F8013B11F003034A
:10C9A00000F02580083AC0F0088051F8043B083AAE
:10C9B00051F804CBA0E80810F5E7121D5CBF51F850
:10C9C000043B40F8043BAFF30080D20724BF11F8CA
:10C9D000013B11F801CB48BF11F8012B24BF00F82F
:10C9E000013B00F801CB48BF00F8012B704710B5A0
:10C9F000203AC0F00B80B1E81850203AA0E8185057
:10CA0000B1E81850A0E81850BFF4F5AF5FEA027C17
:10CA100024BFB1E81850A0E8185044BF18C918C086
:10CA2000BDE810405FEA827C24BF51F8043B40F827
:10CA3000043B08BF7047D20728BF31F8023B48BF0C
:10CA400011F8012B28BF20F8023B48BF00F8012B4A
:10CA5000704702F0FF0343EA032242EA024200F079
:10CA600002B84FF000020429C0F0128010F0030C4D
:10CA700000F01B80CCF1040CBCF1020F18BF00F8D1
:10CA8000012BA8BF20F8022BA1EB0C0100F00DB880
:10CA90005FEAC17C24BF00F8012B00F8012B48BFDE
:10CAA00000F8012B70474FF0000200B51346944682
:10CAB0009646203922BFA0E80C50A0E80C50B1F1F6
:10CAC0002001BFF4F7AF090728BFA0E80C5048BF0A
:10CAD0000CC05DF804EB890028BF40F8042B08BFA8
:10CAE000704748BF20F8022B11F0804F18BF00F8A4
:10CAF000012B704710B5044610F0030F08BF11F06A
:10CB0000030F40F015804FF0013E121FC0F20E805F
:10CB100051F8043BA3EB0E0C2CEA030C1CEACE1CD0
:10CB200008BF40F8043BF0D0A1F1040102F1040277
:10CB3000521E08DB11F8013B002B00F8013BF7D136
:10CB40001146FFF78EFF204610BD704770477047B3
:10CB50007047000010B500F07BFB001D10BD00BF4A
:10CB600021620000004870475C9B002010B5FFF771
:10CB7000F9FF006810BD10B50446FFF7F3FF04602D
:10CB800010BD2DE9F0470D4699469246044600F146
:10CB900024080168880604D5E06921F010012160AD
:10CBA00000E00120A84201DD471B00E00027A16949
:10CBB0007A1902EB0900081AA0612078C00602D495
:10CBC0002046FFF729FC002608E0D4E901211AF8E5
:10CBD00006009047206A401C761C20624E45F4DB1C
:10CBE0002078C0060AD52046FFF716FC06E0D4E9F7
:10CBF000012130209047206A401C2062381EA7F196
:10CC00000107F4DC07E0D4E9012118F8050090479A
:10CC1000206A401C2062281EA5F10105F3DC204695
:10CC2000FFF710FC2078000602D50220BDE8F0874F
:10CC30000120FBE770472DE9FF4F0C461E464FF0E1
:10CC4000FF378BB0D2E90001DDF860800A908A4698
:10CC5000C1F30A5505B93D46002108464FF00000D2
:10CC6000BAF1000F00F4400005DA00EB80004FF449
:10CC7000400101EA50004FEA9059B9F1010F00DD7F
:10CC8000B9460A9850EA4A000ED044F61050A5F270
:10CC9000FF3545432F14B8F1000F1ED07542291EF1
:10CCA0001EDDC9F100021CE0B8F1010F4FF00000D9
:10CCB00001D0302103E0F24305E02154401CB04292
:10CCC000FBDB30460022002121540B99C1F808807B
:10CCD000C1E900200FB0BDE8F08FBD1B6D1CDEE781
:10CCE0004A4600DA694206A800F00AFD06AB93E85E
:10CCF000070003AB83E8070050460A9900F0F2FDF5
:10CD00008DE80700A0F500501F3800900398002D13
:10CD10000ADD42F21F014A460844002303A903909A
:10CD2000684601F05BF809E0A0F500504A461F385C
:10CD3000002303A90390684601F065F88DE8070019
:10CD40000004000C03D04FF0FF30410800E0104613
:10CD5000B8F1000F03D00022009215461EE0751EA8
:10CD600005D400F079FA303262556D1EF9D5B3461C
:10CD70000122084302D000227F1C04E020783028E2
:10CD800001D100227F1E002A099784D01DE0112DB9
:10CD900007DA00F061FA303262556D1C50EA010288
:10CDA000F5D1084302D00098C8B10EE00021681EFA
:10CDB00005E0235C625C63542254401E491C81429E
:10CDC000F7DBAB46A81B401E0990002004F80B00BF
:10CDD0000B98099AC0F80880C0E9002B7AE7112661
:10CDE0004FF0000857E72DE9F04F88460446D21D62
:10CDF00022F0070191B0D1E90001CDE90A0103F069
:10CE00004BFE02460B98C00F01D02D2007E0206892
:10CE1000810701D52B2002E0202101EAC000032A6E
:10CE2000099001D0072A05DB03464146204600F061
:10CE3000D7FB0BE12078800601D5E06900E00620F1
:10CE4000B8F1650F814606D0B8F1660F18D0B8F179
:10CE5000670F70D131E00020B9F1110F009001DBB4
:10CE6000112301E009F101030AAA01A90CA8FFF7A7
:10CE7000E2FEDDE90C70002609F10105834647E07A
:10CE800001204B4600904FF000470AAA01A90CA8C8
:10CE9000FFF7D1FEDDE90DB00C995D46002610B913
:10CEA00009F101000D18B9EB050003D4C0F1FF36FC
:10CEB00009F10105A5EB09002BE0B9F1010F01DA39
:10CEC0004FF001090020B9F1110F0090484601DD33
:10CED000112300E003460AAA01A90CA8FFF7ABFE44
:10CEE000DDE90C704D4600268346207800070AD401
:10CEF000AB4500DA5D4601A8012D04DD411911F8AA
:10CF0000011C302907D04F4502DA17F1040F04DA6B
:10CF1000012082460FE06D1EEEE7002F02DCED1BC4
:10CF20003E4403E0781CA84200DD7D1CB81B00F1E4
:10CF3000010A4FF000472078000703D4AA4501DB1F
:10CF40004FF0FF3A0021B7F1004F0DF143088DF883
:10CF5000431024D002202B23002F01DA7F422D23FF
:10CF60000A21021EA0F1010000DC5FB197FBF1FC79
:10CF700097FBF1F201FB1C7C17460CF1300C08F812
:10CF800001CDEEE7A8F1010003702188090501D564
:10CF9000452100E06521A0F1010800F8011C099875
:10CFA0000FA9A1EB0807FF1D00B10120411901EBFA
:10CFB000EA70A1693844081A401EA0612078C006B2
:10CFC00002D42046FFF728FA099828B1D4E90121B4
:10CFD0009047206A401C20622078C00622D5204657
:10CFE000FFF71AFA1EE0002E04DBB34502DD01A8AC
:10CFF000805D00E03020D4E901219047206A401C88
:10D000002062761CAAF101005FEA000A0AD100F052
:10D010001FF9C0680168405CD4E901219047206A8B
:10D02000401C2062281EA5F10105DCDC07E0D4E9E4
:10D03000012118F8010B9047206A401C2062381E1D
:10D04000A7F10107F3DC2046FFF7FCF9032011B03C
:10D0500041E6000001694A1C02610878704700B58A
:10D060008FB0CDE901310021059105497944CDE921
:10D07000031011466846FFF761FB0FB000BD0000CA
:10D08000E5FFFFFF0A6802F8010B0A607047D1E96B
:10D0900000239A4202D2531C0B601070704710B5E7
:10D0A000436913B1AFF3008001E0FFF7EEF901200F
:10D0B00010BD127800F124010A7000224A7001228A
:10D0C000EDE711684FF0FF32E9E70000074B70B55C
:10D0D0000D467B44FFF7C3FF0446284600F082FB61
:10D0E00010B14FF0FF3070BD204670BDCB3A00004C
:10D0F00010B5436913B1AFF3008001E0FFF73EFACA
:10D10000012010BD128800F1240182840022C28413
:10D110000122EDE711684FF0FF32E9E72DE9F04118
:10D120008046D21D22F007020025D2E90002F5292F
:10D1300015A614D0011E72F1000106DA0023D0EB0F
:10D14000030063EB020211A608E0D8F800108B0779
:10D1500001D50FA602E0490701D50EA6012511460B
:10D16000002408F1240704E000F076F830323A5544
:10D17000641C50EA0102F7D12B4632462146404654
:10D18000BDE8F041FFF7FDBC000000002D000000ED
:10D190002B000000200000002DE9F04791460F46CB
:10D1A00080460446002614F8015B2DB1FFF7D2FC3F
:10D1B0000068405DC007F6D12B2D02D02D2D18D070
:10D1C000641E4A463946204600F04AFA27B13968BB
:10D1D000A14201D1C7F800804FF0020471050BD5C0
:10D1E0004042002803DDFFF7BDFC0460A007BDE856
:10D1F000F08746F48066E4E70028F8DAFFF7B2FC2F
:10D2000004606FF00040F2E770B516460C46054624
:10D21000FFF7A0FC036893F80101012806D0FF2C5A
:10D220000FD8185D68B101202C7070BDD3F80701CC
:10D230003246214603F2071303442846BDE87040F6
:10D2400018474FF0FF3070BD004870475C9B0020CE
:10D25000004870477C9B002030B5B0F10A024FEACD
:10D26000900E71F100034EEA817EB0EB0E0061EB8F
:10D2700091014FEA101E4EEA017E10EB0E0041EBC9
:10D2800011114FEA102E4EEA016E10EB0E0041EB29
:10D2900011214FEA104E4EEA014E10EB0E0041EB09
:10D2A0001141401841F100014FEAD00040EA4170BD
:10D2B0004FEAD10110EB80054FEA810444EA9074F3
:10D2C00044EB01046D1944EB0404521BA3414FF0DD
:10D2D000000348BF0A3200D530BD401C41F10001B7
:10D2E00030BD00002DE9F04F04460D46D21D22F05E
:10D2F000070089B0D0E900974846394603F0CCFBD7
:10D300000246F80F01D02D2307E02068810701D5E0
:10D310002B2302E0202101EAC0038DF820300BB15D
:10D32000012000E00020032A824601D0072A04DB06
:10D330002946204600F054F93FE12078800601D4C8
:10D340000D2500E0E569C7F30A560D2D49DA0021E5
:10D350004FEA175B08464FF00000002F00F4400032
:10D3600007DA00EB80004FF4400100EBD07001EAD7
:10D3700060008115012901DD4FF0FF3100224FEAE5
:10D38000850CBCF1180F06D31346ACF118004FF012
:10D390008052C24003E04FF4801323FA0CF30CF1E7
:10D3A0000C0CBCF1200F04D3ACF1200C09FA0CF0EA
:10D3B00001E007FA0CF000294FF0004801DD18B930
:10D3C0000FE00ED140450CD319EB02095F4121B9A2
:10D3D000404502D19F4329EA0209BBEB175F00D009
:10D3E000761C2088000502D57B48784402E07A4804
:10D3F0007844193808AA302302F80A30037C0AF16D
:10D400000101002E0AF1020A53546A4602DC4FF071
:10D41000300101E04FF031014FF001088DF80010AC
:10D4200002D0A6F2FF3603E059EA470100D06B4E66
:10D43000002D02DC2178090704D54FF002082E21C7
:10D440008DF80110C44600210BE0C7F303433F01F0
:10D45000C35C491C6D1E02F80830052908F101085B
:10D4600001DA002DF1DC00210CE000EB1973491CFE
:10D470001B786D1E082902F808304FEA091908F1D7
:10D48000010801DA002DF0DC21688B0602D516E0D8
:10D49000A8F10108E04505DD02EB080313F8013CA3
:10D4A000302BF5D0B8F1000F09DD02EB080313F8BB
:10D4B000013C2E2B03D1090701D4A8F10108002D4E
:10D4C00005DD3E2102F808106D1E08F10108407CC0
:10D4D000002E02F8080008F1010804DA2D20764237
:10D4E00002F8080002E02B2002F808000A214FF49D
:10D4F0007A70864208F101080BDB96FBF0F33033BB
:10D5000002F8083096FBF0F308F1010800FB1366FF
:10D5100001E0642E0CDB642096FBF0F3303302F85C
:10D52000083096FBF0F308F1010800FB136601E0F8
:10D530000A2E06DB96FBF1F0303002F8080008F105
:10D54000010896FBF1F001FB1060303002F8080092
:10D55000A16908F1010808EB050202EB0A00081AAC
:10D56000A0612078C00602D42046FEF755FF216A4C
:10D5700008AE01EB0A00206204E0D4E9012116F8AC
:10D58000010B9047BAF1010AF7D22078C00602D504
:10D590002046FEF741FF6E4609E016F8010B3E28D3
:10D5A0000FD0D4E901219047206A401C2062B8F1D5
:10D5B0000108F2D22046FEF745FF09B00320BDE87E
:10D5C000F08F206A2844206203E0D4E90121302052
:10D5D00090476D1EEBD3F8E7DD65000002FCFFFF0E
:10D5E0002DE9F0411F46044603260168072A01F48D
:10D5F000006004DB08B116A505E016A503E008B13C
:10D6000015A500E015A521F010002060A069C01E3E
:10D61000A0610FB1401EA0612046FEF7FDFE4FB194
:10D62000D4E9012138469047206A401C2062C01C82
:10D63000206206E0206AFAE7D4E9012115F8010B1F
:10D640009047761EF8D22046FEF7FCFEBDE8F0813A
:10D650004E414E006E616E00494E4600696E660096
:10D660002DE9F05F824615468B4600270AF101043A
:10D67000B9460078302801D09DB113E014F8010BB1
:10D680000127782803D0582801D045B10AE00DB110
:10D69000102D07D1002714F8010B102502E00825F2
:10D6A00000E00A250026B0460EE005FB080005FB59
:10D6B00006F101271FFA80F801EB1046B6F5803F0E
:10D6C00000D3B94614F8010B294600F0B4F800283D
:10D6D000EBDABBF1000F05D00FB1641E00E0544639
:10D6E000CBF80040B9F1000F06D0FFF73BFA02215A
:10D6F0000160C81EBDE8F09F48EA0640FAE7000056
:10D700002DE9F047814616468AB0354878440DC861
:10D710008DE80D0032487844801C03AC0DC884E8C5
:10D720000D0041F69B300844372190FBF1F290FB4D
:10D73000F1F5A5F1800501FB12041B3C02D5644202
:10D74000012000E00020DFF898A080460027FA447E
:10D75000AAF1BE0A0EE0E0070AD03246684607EB9F
:10D76000470101230AEB810100F04DFB8DE8070022
:10D7700064107F1C002CEED1194F7F44AE3F19E09E
:10D78000E80715D007EB04100DF1180A90E80E0019
:10D790008AE80E00C068F04201D19819089032461C
:10D7A000012306A903A800F02EFB03AB83E80700C2
:10D7B0006D10641C002DE3D14FF001033246694621
:10D7C000B8F1000F03A802D000F008FB01E000F060
:10D7D0001AFBC9E90001C9F808200AB0BDE8F087C2
:10D7E0004C630000007B00F0800070477546FFF737
:10D7F0002BFDAE4605006946534620F007008546DE
:10D8000018B020B5FEF7B2FDBDE820404FF000068D
:10D810004FF000074FF000084FF0000B21F0070118
:10D82000AC46ACE8C009ACE8C009ACE8C009ACE85B
:10D83000C0098D4670473A2800D2303820F02002C7
:10D84000412A01D3A2F13700884201D34FF0FF30C3
:10D85000704710B50446AFF300802046BDE8104085
:10D86000FEF723BD4FF0013C50F8042B51F8043B68
:10D870009A4221D1A2EB0C03934313EACC1317D1A4
:10D8800050F8042B51F8043B9A4215D1A2EB0C033B
:10D89000934313EACC130BD150F8042B51F8043BFB
:10D8A0009A4209D1A2EB0C03934313EACC13DBD0C9
:10D8B0004FF00000704700BFD01A01BAB1FA81F1F1
:10D8C00001F0180122FA01F0CB40C1F12001DBB2D6
:10D8D000C0B2C01A2CFA01F3D11A914311EAC31154
:10D8E000E6D170475FEA400C08BF91F0000F4FEAA5
:10D8F0008C234FEAC12243EA51514FEA1C5018BF12
:10D9000000F5F0404FEA300018BF41F000415FEAF7
:10D910006C5C00F02980BCF1FF3F08BF40F0804004
:10D920007047130C06BF12044FF0100C4FF0000CA0
:10D93000130E04BF12020CF1080C130F04BF1201E6
:10D940000CF1040C930F04BF92000CF1020CD30FE6
:10D9500004BF52000CF1010C11464FF00002A0F17F
:10D960001F00A0EB0C00704711F0004F08BF70477C
:10D9700031F000413FF4D5AF0B0C06BF09044FF066
:10D98000100C4FF0000C0B0E04BF09020CF1080C38
:10D990000B0F04BF09010CF1040C8B0F04BF8900AD
:10D9A0000CF1020CCB0F04BF49000CF1010CCCF1BF
:10D9B0002003A0EB0C0022FA03F302FA0CF241EA76
:10D9C000030100F10100704720F07F4C80EA030062
:10D9D00023F07F47ACEB070303F57C5300F00040D6
:10D9E00003F1FF032DE980494FEA154B09B44FEAD3
:10D9F000144325EA0B4E24EA03480FF2042606EBF3
:10DA0000132749083E785FEA320203FB0667C7F531
:10DA1000000707FB06F64FEA54374FEAD64606F1F1
:10DA2000020607FB066CCCF1005C4FEA1C472CEAAF
:10DA3000074C07FB06F40CFB06F504EB15464FEA12
:10DA4000961634BF00204FF000404FEAD13706FB56
:10DA500007FC4FEA1C4C0CFB0BF7D21B03FB0CF72B
:10DA600061EB07010CFB0EF7B0EB074072EB1742BE
:10DA70000CFB08F734BFA2EB0742B2EB074261EBA5
:10DA800017414FEA0C444FEA910706FB07FC4FEAA7
:10DA90001C4C0CFB0BF7B0EBC74072EB573203FB8F
:10DAA0000CF734BFA2EBC742B2EBC74261EB573170
:10DAB0000CFB0EF7B0EBC70072EB57720CFB08F7CC
:10DAC00034BFA2EBC702B2EBC70261EB5771039FF1
:10DAD0004FEA816141EA921104EBCC044FEAD1375D
:10DAE0004FEA826206FB07FC42EA90124FEA80602E
:10DAF0004FEA1C4C0CFB0BF7D21B03FB0CF761EB42
:10DB000007010CFB0EF7B0EB074072EB17420CFB62
:10DB100008F734BFA2EB0742B2EB074261EB1741B3
:10DB20004FEA8C554FEA910704EB9C2406FB07FC57
:10DB30004FEA1C4C0CFB0BF7B0EBC74072EB5732B3
:10DB400003FB0CF734BFA2EBC742B2EBC74261EB59
:10DB500057310CFB0EF7B0EBC70072EB57720CFBA2
:10DB600008F734BFA2EBC702B2EBC70261EB5771F3
:10DB700015EB4C254FEA816141EA92114FEA82622E
:10DB80004FEAD13742EA901206FB07FC44F1000449
:10DB90004FEA80604FEA1C4C0CFB0BF7D21B03FBD7
:10DBA0000CF761EB07010CFB0EF7B0EB074072EBD3
:10DBB00017420CFB08F734BFA2EB0742B2EB074257
:10DBC00061EB174115EB1C154FEA813141EA924197
:10DBD0004FEA823242EA90424FEA80304FEA0C76B6
:10DBE00044F1000448EA03434EEA0B484FF0000EAC
:10DBF000B2EB080C71EB030724BF624639464EEBCB
:10DC00000E0E4FF0000B0018524149414BEB0B0B2D
:10DC1000B2EB080C71EB03077BF1000B24BF6246EB
:10DC200039464EEB0E0E4FF0000B001852414941A1
:10DC30004BEB0B0BB2EB080C71EB03077BF1000B0A
:10DC400024BF624639464EEB0E0E51EA020718BF5A
:10DC500046F0010616EB0E7655F1000254F1000174
:10DC600003D5BDE88901BDE80088BDE88901BDE8AC
:10DC70000048B619524141EB0101A3F1010370477D
:10DC800080807F7E7D7C7B7A7978777676757473F9
:10DC9000727171706F6E6E6D6C6C6B6A6A696868B8
:10DCA000676666656464636362616160605F5F5E4E
:10DCB0005E5D5D5C5C5B5B5A5A59595858575756C4
:10DCC0005655555554545353525252515150505029
:10DCD0004F4F4F4E4E4D4D4D4C4C4C4B4B4B4A4A7B
:10DCE0004A494949484848474747474646464545BF
:10DCF00045444444444343434342424242414141F8
:10DD0000002B9C4630D477002BD01CB54FEA370748
:10DD100003B44FF010004FF01001BAF1000F06D01D
:10DD2000BCF1000FDCBF40F0080040F008014FF0EC
:10DD300000000FBCBDE810400BF1010BBBF1010F5F
:10DD400008BF5FEA170722BF12F1010211F10101BA
:10DD50004FF0004143F1000300F0004043EA0000AF
:10DD60007047F9D35708D0E746EA064613F1400F4B
:10DD70004FEA16461FDD13F1200FDFBF16430A4698
:10DD8000002120335B42BED0C3F1200746EA06469D
:10DD900002FA07F74FEA164646EA0706C3F12007DC
:10DDA00022FA03F201FA07F721FA03F14FF0000318
:10DDB00042EA0702A7E746EA020646EA06464FEAB3
:10DDC000164646EA0106BCBF46EA0646360C4FF048
:10DDD00000034FF000024FF0000194E72DE9804C62
:10DDE0009A46934670B491E8380007C831EA400C6F
:10DDF00048BF34EA430C03D5FFF7E6FDFFF780FF89
:10DE0000F0BCBDE8008C2DE9804C9A46934670B476
:10DE100091E8380007C810F0804F08BF13F0804F1A
:10DE200003D100F005F8FFF76BFFF0BCBDE8008CF4
:10DE300020F07F4780EA030023F07F4C07EB0C03C0
:10DE4000A3F57C5300F00040A3F1FE0392F0000F15
:10DE500000F0B38095F0000F00F077802DE90149C4
:10DE60004FEA11404FEA144621EA004800FB06FC45
:10DE700024EA064708FB06F607FB08F800FB07F74D
:10DE800018EB06484CEB164C4FEA124B18EB0748C0
:10DE90004FEA15464CEB174022EA0B4E0BFB06FCF3
:10DEA00025EA06470EFB06F607FB0EFE0BFB07F7FF
:10DEB0001EEB064E4CEB164C4FF000061EEB074EC9
:10DEC0004CEB174B18EB0B0840F1000018EB0E0B56
:10DED00058EB000840F100008F1A4FF000013CBFE2
:10DEE000C943661B14BFB5EB040C00213CBFC943FA
:10DEF000F61B4FEA17444EEA8E0E27EA04454FEA16
:10DF00001C4704FB07622CEA074C05FB07F70CFBD8
:10DF100005F604FB0CFC16EB074642EB174216EB2A
:10DF20000C4642EB1C421BEB060658EB0202414139
:10DF300046EA9E0601D5BDE80189B619524141EB7A
:10DF40000101A3F10103BDE801894FEA14454FEA3D
:10DF5000114724EA054621EA074C05FB07F406FBB6
:10DF600007F70CFB06F105FB0CFC11EB074144EB3A
:10DF700017444FEA124711EB0C4144EB1C4422EAD0
:10DF8000074C05FB07F206FB07F70CFB06F605FB43
:10DF90000CFC16EB074642EB174216EB0C4642EB25
:10DFA0001C456A1854F1000148BF7047B619524128
:10DFB00041EB0101A3F10103704795F0000F37D049
:10DFC0004FEA11424FEA144721EA024624EA074C7D
:10DFD00002FB07F106FB07F70CFB06F402FB0CFC47
:10DFE00014EB074441EB17414FEA154714EB0C447F
:10DFF00041EB1C4125EA074C02FB07F506FB07F73E
:10E000000CFB06F602FB0CFC16EB074645EB17452E
:10E0100016EB0C4645EB1C42121951F1000148BFAA
:10E020007047B619524141EB0101A3F1010370475A
:10E030004FEA14454FEA114724EA054621EA074C06
:10E0400005FB07F106FB07F70CFB06F24FF0000695
:10E0500005FB0CFC12EB074241EB174112EB0C42A3
:10E0600051EB1C4148BF7047921841EB0101A3F1ED
:10E07000010370470FB4F8B507AD00954FF4007475
:10E08000204602F0B3FF064611A221463046FEF7B5
:10E09000A7F90446C4F5007130192B46069AFEF71D
:10E0A00079F9002806DD204482B23146002002F0D2
:10E0B0005DF907E0502208A10EA0FEF785F911A036
:10E0C000FEF782F9304602F08DFFF8BC5DF814FBD4
:10E0D0004C6F674170703A002E2E5C535953544573
:10E0E0004D5C535953504F52545C737973706F7237
:10E0F000742E63004C6F674572723A2025732C258D
:10E10000640000000000000010B501F0A9FE01F05D
:10E1100047FA002001F0D8FA01F0AAFBBDE8104050
:10E1200001F038BAFEE730B500231AE0CD5C2C09C7
:10E1300005F00F053034392C03D9E41D00F81340E5
:10E1400001E000F813403035ECB2392C04D900EB73
:10E150004305E41D6C7002E000EB43056C705B1C32
:10E160009BB29342E2D330BD10B5022000F0C2FB57
:10E17000012805D1022000F0D9FA022000F0C0FCED
:10E18000082000F0B7FB01280FD1082000F0CEFADC
:10E19000D52206A10AA0FEF717F90DA0FEF714F983
:10E1A000BDE81040082000F0ABBC10BD2E2E5C5323
:10E1B000595354454D5C444D415C646D612E630080
:10E1C0004C6F674572723A2025732C25640000005D
:10E1D000444D41315F5445312100000010B52020ED
:10E1E00000F088FB012805D1202000F09FFA2020B4
:10E1F00000F086FC802000F07DFB01280FD18020FC
:10E2000000F094FAEB2206A10AA0FEF7DDF80DA0BB
:10E21000FEF7DAF8BDE81040802000F071BC10BDB8
:10E220002E2E5C53595354454D5C444D415C646DF6
:10E23000612E63004C6F674572723A2025732C255E
:10E2400064000000444D41315F544532210000001C
:10E2500010B54FF40074204600F04CFB012805D1A6
:10E26000204600F063FA204600F04AFC4FF40064B8
:10E27000204600F03FFB012810D1204600F056FA5E
:10E2800040F2011206A10BA0FEF79EF80DA0FEF7CA
:10E290009BF82046BDE8104000F032BC10BD0000E5
:10E2A0002E2E5C53595354454D5C444D415C646D76
:10E2B000612E63004C6F674572723A2025732C25DE
:10E2C00064000000444D41315F544533210000009B
:10E2D00010B54FF40054204600F00CFB012805D186
:10E2E000204600F023FA204600F00AFC4FF40044D8
:10E2F000204600F0FFFA012810D1204600F016FA5F
:10E3000040F2171206A10BA0FEF75EF80DA0FEF773
:10E310005BF82046BDE8104000F0F2BB10BD0000E5
:10E320002E2E5C53595354454D5C444D415C646DF5
:10E33000612E63004C6F674572723A2025732C255D
:10E3400064000000444D41315F5445342100000019
:10E3500010B54FF40034204600F0CCFA012805D166
:10E36000204600F0E3F9204600F0CAFB4FF40024F9
:10E37000204600F0BFFA012810D1204600F0D6F95F
:10E3800040F22D1206A10BA0FEF71EF80DA0FEF71D
:10E390001BF82046BDE8104000F0B2BB10BD0000E5
:10E3A0002E2E5C53595354454D5C444D415C646D75
:10E3B000612E63004C6F674572723A2025732C25DD
:10E3C00064000000444D41315F5445352100000098
:10E3D00010B54FF40014204600F08CFA012805D146
:10E3E000204600F0A3F9204600F08AFB4FF4000419
:10E3F000204600F07FFA012810D1204600F096F95F
:10E4000040F2431206A10BA0FDF7DEFF0DA0FDF7C1
:10E41000DBFF2046BDE8104000F072BB10BD0000DD
:10E420002E2E5C53595354454D5C444D415C646DF4
:10E43000612E63004C6F674572723A2025732C255C
:10E4400064000000444D41315F5445362100000016
:10E4500010B54FF00074204600F04CFA012805D1A9
:10E46000204600F063F9204600F04AFB4FF00064BC
:10E47000204600F03FFA012810D1204600F056F95E
:10E4800040F2591206A10BA0FDF79EFF0DA0FDF76B
:10E490009BFF2046BDE8104000F032BB10BD0000DD
:10E4A0002E2E5C53595354454D5C444D415C646D74
:10E4B000612E63004C6F674572723A2025732C25DC
:10E4C00064000000444D41315F5445372100000095
:10E4D00010B5124C204600F00DFA012805D1204657
:10E4E00000F024F9204600F00BFB0C4CA41D204644
:10E4F00000F000FA012810D1204600F017F940F290
:10E500006F1207A10BA0FDF75FFF0EA0FDF75CFFE8
:10E510002046BDE8104000F0F3BA10BD0200001024
:10E520002E2E5C53595354454D5C444D415C646DF3
:10E53000612E63004C6F674572723A2025732C255B
:10E5400064000000444D41325F5445322100000018
:10E5500010B5124C204600F0CDF9012805D1204617
:10E5600000F0E4F8204600F0CBFA0C4C6034204672
:10E5700000F0C0F9012810D1204600F0D7F840F291
:10E58000851207A10BA0FDF71FFF0EA0FDF71CFFD2
:10E590002046BDE8104000F0B3BA10BD20000010C6
:10E5A0002E2E5C53595354454D5C444D415C646D73
:10E5B000612E63004C6F674572723A2025732C25DB
:10E5C00064000000444D41325F5445322100000098
:10E5D00010B5124C204600F08DF9012805D12046D7
:10E5E00000F0A4F8204600F08BFA0D4C204600F015
:10E5F00081F9012810D1204600F098F840F29B12D2
:10E6000008A10DA0FDF7E0FE0FA0FDF7DDFE2046FE
:10E61000BDE8104000F074BA10BD00000002001008
:10E62000000800102E2E5C53595354454D5C444D48
:10E63000415C646D612E63004C6F674572723A20D5
:10E6400025732C2564000000444D41325F5445334E
:10E650002100000010B5224C204600F04BF90128A3
:10E6600005D1204600F062F8204600F049FA1D4C22
:10E67000204600F03FF901280ED1204600F056F860
:10E6800040F2B11218A11DA0FDF79EFE1FA0FDF7DC
:10E690009BFE204600F034FA1F4C204600F02AF979
:10E6A000012805D1204600F041F8204600F028FA64
:10E6B0001A4C204600F01EF9012810D1204600F027
:10E6C00035F84FF4DF7208A10CA0FDF77DFE14A011
:10E6D000FDF77AFE2046BDE8104000F011BA10BDEB
:10E6E00000200010008000102E2E5C53595354451A
:10E6F0004D5C444D415C646D612E63004C6F674519
:10E7000072723A2025732C2564000000444D41327A
:10E710005F54453421000000000002100000081082
:10E72000444D41325F54453521000000C10002D5FF
:10E73000024908607047024948607047040402407B
:10E7400000000240002904D0016841F0010101608D
:10E75000704701684FF6FE7211400160704700007B
:10E760002DE9F0478CB00446DDE914980D461746B4
:10E770009A46072C04D20121084601F015F903E05E
:10E780000121022001F010F9184E56F8240000F083
:10E7900031F801950297CDF80CA000250495059558
:10E7A0008020069007950895CDF8249040010A90A6
:10E7B0000B9556F8240001A900F0B8F80C4810F8A1
:10E7C00024008DF800008DF801808DF802500120A2
:10E7D0008DF80300684601F001F856F82400012284
:10E7E000022100F099F80CB0BDE8F0879C000020F1
:10E7F0006038020801684FF6FE7211400160002186
:10E80000016041608160C1603649364A08399042F2
:10E8100004D1486840F00F0048607047314A143214
:10E82000904204D1486840F0F000486070472D4A9B
:10E830002832904204D1486840F4706048607047C4
:10E84000284A3C32904204D1486840F47040486005
:10E850007047244A5032904204D1486840F47020F6
:10E86000486070471F4A6432904204D1486840F4BF
:10E870007000486070471B4A7832904204D1486863
:10E8800040F0706048607047174A111F904204D1F1
:10E89000086840F00F0008607047134A1432904235
:10E8A00004D1086840F0F000086070470E4A283232
:10E8B000904204D1086840F47060086070470A4ACA
:10E8C0003C32904204D1086840F4704008607047C0
:10E8D000054A50329042FAD1086840F4702008602E
:10E8E000704700000800024008040240406880B2FF
:10E8F0007047000002460020D10002D50449096893
:10E9000001E004490968114200D00120704700006D
:10E910000004024000000240002A03D002680A43BB
:10E920000260704702688A430260704730B502682F
:10E9300047F6F0739A430C6A8B682343D1E9044588
:10E940002C4323438C692343CC6923434C6A2343E0
:10E950008C6A234313430360CA6842600A6882607A
:10E960004968C16030BD416070470721022000F056
:10E97000FBBD704770B5044603F0D2FF01280CD0F0
:10E98000094D6888844203D3B4FBF0F003F070FAB9
:10E990006888B4FBF0F100FB11444FF47A706043D7
:10E9A000BDE8704000F002B8F400002070B50546E4
:10E9B0001148854208D90546612210A116A0FDF72D
:10E9C00003FD19A0FDF700FD00214FF0E02674695A
:10E9D000164800784543B369B2699A42FCD003D225
:10E9E000A3EB0200014403E0A4EB0200184401443D
:10E9F0001346A942F0D370BDE3388E032E2E5C532C
:10EA0000595354454D5C5359535449434B5C7379A6
:10EA1000737469636B2E63004C6F674572723A20A2
:10EA200025732C256400000000000000F400002085
:10EA300070B505460C467B2001F03EF8012804D154
:10EA400022461EA12846FEF755F87C2001F034F836
:10EA5000012804D122461CA12846FEF74BF87D2050
:10EA600001F02AF8012804D122461AA12846FEF70F
:10EA700041F87E2001F020F8012804D1224619A196
:10EA80002846FEF737F87C2001F016F888B97D207B
:10EA900001F012F868B97E2001F00EF848B97A202A
:10EAA00001F00AF8012804D1224612A12846FEF7F7
:10EAB00021F8BDE8704000F0A1BF0000D6D8C9CF52
:10EAC000B5E7C6F4B6AF0000C8EDB8B4CEBBC6F427
:10EAD000B6AF0000B6C0C1A2BFB4C3C5B9B7C6F4D3
:10EAE000B6AF0000B4B0BFDABFB4C3C5B9B7C6F49F
:10EAF000B6AF0000D3B2B8B4CEBBC6F4B6AF000018
:10EB000030B46A49B0F1007F01F1300271D036DCD7
:10EB1000B0F5005F6ED018DC80287AD00ADC0228BD
:10EB20006DD0082870D0202868D14868002865D0AA
:10EB300030BC0047B0F5007F71D0B0F5006F5DD1FB
:10EB4000906800285AD030BC0047B0F5002F77D02D
:10EB50000ADCB0F5004F6ED0B0F5003F4ED1086929
:10EB600000284BD030BC0047B0F5001F6DD0B0F589
:10EB7000000F43D15069002840D030BC00474C4CB6
:10EB8000031BA0427CD01ADC4A4CA0EB0403A04239
:10EB90006CD00BDCB0F1006F61D0A0F18050801E12
:10EBA0002CD1C86900287FD030BC0047182B62D018
:10EBB000782B79D1106A002876D030BC0047B3F5A5
:10EBC000FC4F67D00ADCB3F5C06F5ED0B3F5F05FE1
:10EBD0006AD1886A002867D030BC0047B3F5FF3F90
:10EBE0005DD03548C3425FD1D06A00285CD030BCCC
:10EBF00000472FE018E00CE001E005E054E0086871
:10EC0000002851D030BC0047106800284CD030BCE0
:10EC100000475068002847D030BC0047FFE78868AD
:10EC2000002841D030BC0047C86800283CD030BC28
:10EC3000004705E0FFE7D068002835D030BC00472A
:10EC40001069002830D030BC0047486900282BD01C
:10EC500030BC00478869002826D030BC0047906946
:10EC6000002821D030BC00470AE0FFE7D069002827
:10EC70001AD030BC0047086A002815D030BC0047C5
:10EC8000486A002810D030BC0047506A00280BD0DA
:10EC900030BC0047906A002806D030BC0047C86AE4
:10ECA000002801D030BC004730BC7047443F0020F2
:10ECB00000020010080000100002F8FF10B5144612
:10ECC00000290BD0012919D04E2215A119A0FDF75A
:10ECD0007BFB1CA0FDF778FB204610BD224951F8B4
:10ECE000202042B143220EA112A0FDF76DFB1FA010
:10ECF000FDF76AFBF0E741F82040EDE71A493031B3
:10ED000051F8202042B14A2205A10AA0FDF75CFB80
:10ED10001DA0FDF759FBDFE741F82040DCE70000CC
:10ED20002E2E5C53595354454D5C444D415C646DEB
:10ED3000612E63004C6F674572723A2025732C2553
:10ED400064000000446D6154652043616C6C626135
:10ED5000636B202265497271547970652220657257
:10ED6000726F722100000000443F0020446D615426
:10ED7000632043616C6C6261636B207265706561D6
:10ED80007420726567210000446D61546520436101
:10ED90006C6C6261636B2072657065617420726572
:10EDA0006721000010B5012000F0AAF828B1012069
:10EDB00000F09AF8012000F0B7FBBDE810400120F8
:10EDC00000F098B830B591B00A240E4D55F82400E3
:10EDD00000F0A0F888B155F8240000F085F8402133
:10EDE00001A8FDF760FE234607A2402101A8FDF718
:10EDF000F7FA55F8240000F097FB641C0F2CE5DDB2
:10EE000011B030BDE4380208455854492564204902
:10EE10005251210010B5022000F072F8012805D1EE
:10EE2000022000F061F8022000F07EFBBDE81040F7
:10EE3000022000F05FB810B5042000F061F828B19E
:10EE4000042000F051F8042000F06EFBBDE81040F3
:10EE5000042000F04FB810B5082000F051F8012848
:10EE600005D1082000F040F8082000F05DFBBDE867
:10EE70001040082000F03EB810B5102000F040F817
:10EE800028B1102000F030F8102000F04DFBBDE854
:10EE90001040102000F02EB830B591B005240E4D72
:10EEA00055F8240000F036F888B155F8240000F039
:10EEB0001BF8402101A8FDF7F6FD234607A24021DB
:10EEC00001A8FDF78DFA55F8240000F02DFB641C15
:10EED000092CE5DD11B030BDE4380208455854492D
:10EEE0002564204952512100014908607047000003
:10EEF00014040140014908607047000014040140F7
:10EF000001460020024A12680A4200D001207047E0
:10EF10001404014001460020054A12680A40044BCF
:10EF200014331B680B4202D0002A00D00120704726
:10EF30000004014070B500F0CFF80024094D05EB46
:10EF4000C42000F063F8641CE4B2002CF7D006483B
:10EF500000214160C16000F055FEBDE8704000F046
:10EF600099B8000000F80708280B00200FB4F8B586
:10EF700007AD00954FF40074204602F037F80646BE
:10EF800011A221463046FDF72BFA0446C4F5007164
:10EF900030192B46069AFDF7FDF9002806DD2044BE
:10EFA00082B23146002001F0E1F907E08B2208A18E
:10EFB0000EA0FDF709FA11A0FDF706FA304602F09F
:10EFC00011F8F8BC5DF814FB4C6F674572723A009B
:10EFD0002E2E5C53595354454D5C535953504F5248
:10EFE000545C737973706F72742E63004C6F674555
:10EFF00072723A2025732C25640000000000000086
:10F000000149C860704700000020024070B5054605
:10F010004FF43026304600F06BF8042811D1094C2B
:10F02000206940F0020020616561206940F04000E5
:10F030002061304600F05CF8216941F6FD72114014
:10F04000216170BD0020024004200849CA68D2072F
:10F0500001D001207047CA68520701D502207047CD
:10F06000C968C906FBD50320704700000020024094
:10F0700001460020064A012904D0D2680A4200D085
:10F0800001207047D169C907FBD0012070470000FB
:10F09000002002400248016941F08001016170478F
:10F0A00000200240F0B506460D464FF400573846A2
:10F0B00000F01EF804280CD1064C206940F0010035
:10F0C00020613580384600F013F82169BA1E1140DE
:10F0D0002161F0BD0020024003480249416003491C
:10F0E000416070472301674500200240AB89EFCDA6
:10F0F00000B50346FFF7A8FF02E0FFF7A5FF5B1E80
:10F10000012801D1002BF8D1002B00D1052000BD32
:10F110002DE9F0410022CC7804F00F03E40601D57C
:10F120008C7823430C784FF00F0714F0FF0F4FF04B
:10F13000010C1CD005680CFA02F40E882640A64289
:10F1400011D1960007FA06F825EA080503FA06F831
:10F1500048EA0505CE78282E02D0482E02D002E0DB
:10F16000446100E00461521C082AE4D305600A8867
:10F17000FF2A1ED94568002202F108060CFA06F49F
:10F180000E882640A64210D1960007FA06F825EA16
:10F19000080503FA06F848EA0505CE78282E00D1BE
:10F1A0004461CE78482E00D10461521C082AE3D372
:10F1B0004560BDE8F08100000EB50F4A126800926C
:10F1C0000D4A121D126801920B4A0832126802920F
:10F1D00000290BD0012904D00C226946FEF7A3FFB9
:10F1E0000EBD0C226946FEF79EFF0EBD0C2269463D
:10F1F000FDF780FC0EBD0000E8F7FF1F0022028033
:10F20000827001460322014800F0F3BC009001081F
:10F2100010B5F821FDF725FCBDE81040F8220249A1
:10F22000024800F0E6BC00002A0600200088010821
:10F23000F8B504460D4616460B48012150F8240047
:10F2400000F0CEFB08481C3030F81500ADF8000087
:10F250008DF8036003208DF802000448694650F8D9
:10F260002400FFF755FFF8BD98380208CC000020B5
:10F27000162204A10DA0FDF7A7F810A0FDF7A4F831
:10F28000FEE700002E2E5C53544D33324631307869
:10F290005F46574C69625C7372635C73746D3332A2
:10F2A000663130785F69742E630000004C6F6745EB
:10F2B00072723A2025732C25640000004861726444
:10F2C0004661756C745F48616E646C657221000004
:10F2D00002494AF6AA20086070470000003000404A
:10F2E00010B504462046FFF789FF2046BDE81040D0
:10F2F00000F048BD002140F8191F41608160C160E5
:10F300000161416119381921FDF7ABBB7CB5044699
:10F310003E4800F097F82046FFF77AFF5B20207008
:10F32000302060703120A070E070207CFF2809D16F
:10F3300004F1100040210546FDF793FB34A1284657
:10F34000FDF7CDFA94F85000FF2809D104F15000E0
:10F3500040210546FDF785FB2FA12846FDF7BFFAA2
:10F3600094F89000FF2809D104F19000402105464F
:10F37000FDF777FB29A12846FDF7B1FA94F8D000F4
:10F38000FF2809D104F1D00010210546FDF769FBE3
:10F3900026A12846FDF7A3FA94F8E000FF2816D02E
:10F3A000A8B12649264800F069FC94F8F000FF282F
:10F3B00018D0B8B121492248103100F06CFC5D2012
:10F3C00084F8F7002046BDE87C4000F0E3BC04F17F
:10F3D000E00010210546FDF744FB14A12846FDF787
:10F3E0007EFAE2E70020C4F8F000A4F8F4000090F0
:10F3F00001900A22694641F6583001F0DDFB69466A
:10F4000004F1F000FDF76BFAD9E7000024020020B8
:10F410002F41424D0000000041424D0053686F7083
:10F420003334343739343734390000003132312E37
:10F43000352E3231372E3235320000000A070020D7
:10F440001600002000210180418081804FF48061FE
:10F45000801DFDF706BB00002DE9F0418388161DD5
:10F4600033444FF48067BB4202D30120BDE8F081F2
:10F4700045881223841D2B5543885B1CC3F3090365
:10F480004380458834232B5543885B1CC3F3090311
:10F49000438000230BE011F8015BB0F802C00CF8C8
:10F4A000045045886D1CC5F3090545805B1C9342DB
:10F4B000F1DB4288562111554188491CC1F30901ED
:10F4C00041804288782111554188491CC1F30901C6
:10F4D00041808188314481808188B94209D3FFF716
:10F4E000B1FF432204A10BA0FCF76EFF0DA0FCF7B7
:10F4F0006BFF0020BAE700002E2E5C535953544591
:10F500004D5C5359534C49425C7379736C69622E5C
:10F51000630000004C6F674572723A2025732C25FA
:10F52000640000000000000070B5064600204FF0A7
:10F53000804101F06FFB04460D46304603F0E2FEC9
:10F5400001F068FB22462B4603F002FD03F094FE17
:10F55000044951F82000002802D0BDE8704000475F
:10F5600070BD0000A43F0020044A52F82000C26889
:10F57000034B33F811104A40C2607047CC000020A2
:10F58000B438020801F038F9FFF7EFF9642002F00F
:10F590006FFCF7E7102207210220FFF749BE0000A9
:10F5A00070B514221149124800F023FB0F4C4FF0A4
:10F5B000503000252268011182420FD122698A420F
:10F5C0000CD121890BA0FEF755FD1448616800F0AD
:10F5D000DFFA2581BDE8704000F014BB2060216196
:10F5E0002581BDE87040FFF7A5BC0000280B002076
:10F5F00000F00708B1BEB5D8C8D5D6BEB4E6B4A2EF
:10F60000D2E7B3F6A3BA2564B4CE202E0D0AB1BE5C
:10F61000B5D8C8D5D6BE3A200000000000F80708CB
:10F62000FEE70000002906D0034A02EB8002926840
:10F63000891A00F015B870472C00002010B5044658
:10F64000204600F05FF8411C05D0044901EB84011D
:10F650008968084410BD002010BD00002C00002067
:10F6600070B5134A13181B7E002B12D0114B53F8A0
:10F6700020308B421AD90F4B083B53F82030B1FB96
:10F68000F3F102EB8002106930F811300020002401
:10F6900008E011688847012070BD15690E1825F82B
:10F6A0001640401C9842F8DB002070BD022070BD5F
:10F6B0002C0000201C38020801E000F8011B521E3B
:10F6C000531CFAD17047000070B504460B480C4E2D
:10F6D000002150F8240006EB840542002869FFF75A
:10F6E000EBFF06480021103050F82420A868FFF7EF
:10F6F000E3FF01203119087670BD00000C380208C4
:10F700002C0000202DE9F04105460F460024DFF8CB
:10F71000888008EB0500007E002803D1D8F800108F
:10F72000284688474FF0FF32FFB11C4E56F825009F
:10F73000B7FBF0F3B7FBF0F100FB117000B15B1CFD
:10F740001648083850F82510491E002921DB08EB1F
:10F750008507386930F811C0BCF1000F08D00024CB
:10F760009C4213D1002298B20AE01046BDE8F08115
:10F77000641CF5E73C6901EB020C24F81C00521CE8
:10F780009A42F7D356F825004843EFE7491E00296F
:10F79000E0DA1046EAE700002C00002014380208E6
:10F7A00010B5002200210A4B0A4C53F8203004EB1C
:10F7B000800005E0046934F8114004B1521C491C72
:10F7C0008B42F7D864204243B2FBF3F0C0B210BDC5
:10F7D0000C3802082C0000207047000070B50F2381
:10F7E000C27801260178002A1ED0144A126802F459
:10F7F000E062C2F5E062120AC2F10404D340457827
:10F80000A54082781A402A43120101F1E02181F8D3
:10F810000024007800F01F018E404009800000F1B4
:10F82000E020C0F8006170BD01F01F00864048096B
:10F83000800000F1E020C0F8806170BD0CED00E0B8
:10F840000249084302490860704700000000FA05B9
:10F850000CED00E0024A114001430248016070478C
:10F8600080FFFF1F08ED00E04FF48030FFF742BB40
:10F8700030B5A1B02448FCF7A7FD2448FCF7A4FD4F
:10F88000234C2448211D00F018FA224B0B2225336B
:10F89000002121A0FCF798FD1E481930054600F014
:10F8A00073F829461B4800F0FDF929461FA0FCF714
:10F8B0008BFDA17821A03039FCF786FD0121154888
:10F8C000FFF77AFC134A182121A0FCF77DFD1148AF
:10F8D0000B2131300446FFF7ABF822460B2121A063
:10F8E000FCF772FD0848FCF76FFD802101A8FDF7C9
:10F8F000DAF8234620A2802101A8FCF771FD01A8B7
:10F9000000F07CFF21B030BD743A0208B83A02081A
:10F910002A060020E70100200D0A426F6F74B0E64E
:10F92000B1BE203A20252A2E2A7300000D0A41502C
:10F930005020B0E6B1BE203A202573000D0A527562
:10F940006E4170704E756D3A204150502564000034
:10F950000D0AC9E8B1B8B1E0BAC5203A20252E2A6F
:10F96000730000000D0AD6D8C6F4D4ADD2F2203A06
:10F9700020252E2A73000000D6D8C6F4D4ADD2F2CA
:10F980003A25732E000000000021016041600181D2
:10F9900081720B2201A1FDF7ADB800004E6F7620F9
:10F9A0003232203230323300054A002903D0516907
:10F9B00001435161704751698143516170470000B3
:10F9C00000100240054A002903D0D1690143D161EA
:10F9D0007047D1698143D161704700000010024037
:10F9E000054A002903D091690143916170479169EB
:10F9F0008143916170470000001002400248416A53
:10FA000041F08071416270470010024010B5264AF3
:10FA1000516801F00C01254B002927D0042927D07B
:10FA2000082927D00360516801F0F0010909204B33
:10FA30005C5C0168E1404160546804F4E064240ABD
:10FA40001C5D21FA04F48460546804F46054E40AF0
:10FA50001B5DD940C160526802F44042920B144BC6
:10FA60001B1F9A5CB1FBF2F1016110BD0360DAE784
:10FA70000360D8E7516801F47011536803F48033D0
:10FA8000022404EB914133B153689B0307D5094B22
:10FA900059430160C7E7074B59430160C3E7034B74
:10FAA00059430160BFE700000010024000127A00D5
:10FAB0000001002000093D00034600205909094AC1
:10FAC00001290AD002290AD0516A03F01F0201233A
:10FAD00093400B4200D0012070471168F5E7116A8E
:10FAE000F3E700000010024010B5022000F01AF801
:10FAF00000280DD04FF40030FFF7FCF9022000F091
:10FB000009F800F03DF8BDE81040022000F0A6B86A
:10FB100010BD000002490A8882430A807047000035
:10FB20000428004006490988C2B21140044A121F45
:10FB30001288024202D009B10120704700207047AC
:10FB40000428004010B50120FFF7ECFF38B1012078
:10FB5000FFF7E0FF00F014F8012000F07FF802202A
:10FB6000FFF7E0FF002809D00220FFF7D3FF00F0E5
:10FB700007F8BDE81040022000F070B810BD00008A
:10FB8000024801888906FCD570470000042800401F
:10FB90002DE9F04105460E464FF40067384601F066
:10FBA00025FA8046C6F3CF240BE03A464146284664
:10FBB00000F01FF83A464146002000F0D7FB05F55B
:10FBC0000065641EA4B2F0D239464046FCF749FFF6
:10FBD000C6F30A0422464146284600F00AF82246A7
:10FBE0004146002000F0C2FB4046BDE8F04101F074
:10FBF000F9B903E010F8013B01F8013B521E92B243
:10FC0000F8D2704710B5054C2046FFF7FFF92046A3
:10FC1000BDE810401422024900F096BE00F007082B
:10FC2000280B00204FF48065284601F0DFF90446D8
:10FC3000214605A0FEF71EFA204601F0D3F9642004
:10FC400002F016F9F0E70000527332333220726589
:10FC500063646174613A2573202E0000064901280F
:10FC600005D0022807D18868002804D000474868DA
:10FC7000002800D000477047E800002070B5044617
:10FC80000D461021601CFCF7ECFE2946601CBDE807
:10FC90007040FCF724BE10B504460846FCF712FE7F
:10FCA000608210BD10B504460B2204F11900FCF768
:10FCB00021FF002084F8250010BD10B504460B225A
:10FCC00004F12500FCF716FF002084F8310010BD78
:10FCD000AFF300800CB50022019200922748016822
:10FCE00041F4803101604FF4A063016801F40031F8
:10FCF00000910199491C0191009911B9019999420A
:10FD0000F3D10168890302D50121009100E000923E
:10FD10000099012930D11A490A6842F010020A609C
:10FD20000A6822F003020A600A6842F002020A60CE
:10FD30004168416041684160416841F480614160CF
:10FD4000416821F47C114160416841F4E81141604F
:10FD5000016841F08071016001688901FCD541684A
:10FD600021F003014160416841F0020141604168B6
:10FD7000C1F381010229FAD10CBD0000001002403C
:10FD80000020024001460322014800F0DDBD0000D2
:10FD9000009001080146F822014800F0D5BD00009E
:10FDA000008801081CB500F027FD01F019FFFEF7DF
:10FDB000ABF900F021FD0F480121CDE900100A0246
:10FDC00000230DA10F4802F07BFD0A481F21001DF2
:10FDD000CDE90010002380220BA10D4802F070FD38
:10FDE00004480838406802F07BF8BDE81C4001F088
:10FDF00033BF000008000020527332333254617365
:10FE00006B00000025FC01084C65645461736B00B5
:10FE100085F501084FF0E021042804D0086920F09E
:10FE2000040008617047086940F0040008617047E9
:10FE300010B502F075FD01280CD002F04DFA07480C
:10FE4000416811F1020F01D3002141604168491C52
:10FE5000416010BDBDE8104000F0CEBCF4000020B1
:10FE600010B50420FFF7D6FF0C480D490D4A006875
:10FE7000B0FBF1F31370B0FBF1F142F210704143AB
:10FE80000A2050804FF0E020026942F00202026135
:10FE90004161016941F00101016110BD10010020C3
:10FEA00040420F00F400002010B50F48016841F0F7
:10FEB0000101016041680D4A1140416001680C4A2E
:10FEC00011400160016821F480210160416821F442
:10FED000FE0141604FF41F018160FFF7F9FE054903
:10FEE0004FF00060086010BD001002400000FFF8F5
:10FEF000FFFFF6FE08ED00E071B605480168054A0F
:10FF000001F4E06111430160BFF34F8FFEE7000091
:10FF10000CED00E00400FA0510B501218C07204625
:10FF200000F073F8012808D10121204600F06AF89A
:10FF3000BDE81040002000F075B810BD10B5084CA9
:10FF40000121204600F061F8012808D10121204656
:10FF500000F058F8BDE81040012000F063B810BD73
:10FF60000004004010B5084C0121204600F04DF877
:10FF7000012808D10121204600F044F8BDE81040D6
:10FF8000022000F04FB810BD0008004010B5084C2A
:10FF90000121204600F039F8012808D1012120462E
:10FFA00000F030F8BDE81040032000F03BB810BD71
:10FFB000000C004010B5084C0121204600F025F847
:10FFC000012808D10121204600F01CF8BDE81040AE
:10FFD000042000F027B810BD0010004010B5084CF8
:10FFE0000121204600F011F8012808D10121204606
:10FFF00000F008F8BDE81040052000F013B810BD6F
:020000040802F0
:1000000000140040C9430182704702460020138A51
:100010000B4092890A40002B02D0002A00D0012018
:1000200070470000034951F82000002800D0004725
:1000300070470000F83F0020014901200870704718
:100040004C00002001490120487070474C000020FE
:1000500001490120887070474C00002001490120AF
:10006000C87070474C00002070B51C4C40F2244111
:10007000204600F0ACFAA0B1194D0021686AFEF7E5
:1000800061FB2088201D0088686AFEF72FFCC0F500
:10009000807082B21349032000F036FB032000F089
:1000A0006BF840F225552946204600F090FA18B129
:1000B0002946204600F066FA40F227752946204678
:1000C00000F085FA20B100222946204600F09FFA70
:1000D0002046BDE87040402100F050BA004C00407E
:1000E0009C000020443D00202DE9F0411F4D40F2CE
:1000F0002551284600F06BFA1D4C002658B1AA88FD
:100100002168481C20601B484254216846542068DE
:10011000FF2800DB266040F224473946284600F0DD
:1001200056FA88B12888A8882068124982B204202B
:1001300000F0EAFA4FF480710E48FCF7B4FC266038
:100140003946284600F01EFA40F227742146284618
:1001500000F03DFA002806D021462846BDE8F041CF
:10016000002200F054BABDE8F081000000500040C9
:1001700048000020443E00202DE9F0410446104D87
:10018000104E0021285D56F82000FEF7DBFA05F13D
:100190000A0705F1280037F8141050F82400FCF77E
:1001A00060FC285D37F8141056F82000FEF7DBFBE2
:1001B000285D012156F82000BDE8F041FEF7C2BAE3
:1001C000283802089C0000202DE9F04387B004463F
:1001D0000D461646984601210846FFF701FC5F4888
:1001E0001822015D401F005DFFF722F85B480422E2
:1001F0000A30015D401F005DFFF71AF85848002CD7
:100200007ED050F824000121FFF7DCFB0295002589
:10021000ADF80C50ADF80E50ADF81050ADF81450CC
:10022000ADF812604D4E02A90F3656F8240000F0CA
:1002300009FA56F824004FF4587100F09FF9BDF800
:10024000120006F11409000721D5042C1FD056F81E
:1002500024000122802100F0A9F9414F0095019569
:10026000183F59F82410385D10230022FEF778FA61
:1002700006F12400002150F82420385DFEF71EFD11
:100280003848012150F82420385DFEF717FDBDF8ED
:100290001200400759D532481038005D8DF818001B
:1002A0008DF819808DF81A5001208DF81B0006A8D2
:1002B000FFF794FA56F82400012240F2244100F09E
:1002C000A6F9042C3BD056F824000122402100F06E
:1002D0006DF9CDE90058224859F824101430A0F1E6
:1002E000280550F82420285D0023FEF739FA05F18F
:1002F0000A001D4F30F81410285D57F8200000E068
:1003000018E0FEF730FB17480021103050F8242089
:10031000285DFEF7D3FC13480121203050F824203B
:10032000285DFEF7CBFC285D012157F82000FEF781
:1003300009FA0AE000680121FFF752FB66E7012293
:1003400040F22551306900F062F956F8240001218D
:1003500000F020F907B0BDE8F08300005500002050
:100360003C380208003A00209C0000202DE9F047AC
:10037000044688461646B8F1000F23D0002E21D03F
:10038000042C21D01D4FDFF878900021385D59F8FA
:100390002000FEF7D7F91B4D00202855385D59F88D
:1003A0002000C0F80C80385D314659F82000FEF777
:1003B000DAFA385D012159F82000FEF7C3F9285D0B
:1003C0000028FCD0BDE8F08700250E4F40211837EB
:1003D000386900F0F5F80EE018F8051057F8240019
:1003E00000F08EF957F82400402100F0E9F80028C9
:1003F000F8D06D1CADB2B542EED3E3E72438020865
:100400009C0000204C00002070B51B4C40F22441A1
:10041000204600F0DCF8A0B1184D00212869FEF755
:1004200091F92088201D00882869FEF75FFAC0F541
:10043000807082B21249002000F066F90020FFF7B8
:100440009BFE40F225552946204600F0C0F818B121
:100450002946204600F096F840F2277529462046A6
:1004600000F0B5F8002806D029462046BDE87040C7
:10047000002200F0CCB870BD003801409C00002084
:10048000443A002070B51B4C40F22441204600F055
:100490009EF8A0B1184D00216869FEF753F9208835
:1004A000201D00886869FEF721FAC0F5807082B2CD
:1004B0001249012000F028F90120FFF75DFE40F20B
:1004C00025552946204600F082F818B129462046D5
:1004D00000F058F840F227752946204600F077F8DA
:1004E000002806D029462046BDE87040002200F0D2
:1004F0008EB870BD004400409C000020443B0020AA
:1005000070B51B4C40F22441204600F060F8A0B1C9
:10051000184D0021A868FEF715F92088201D0088D5
:10052000A868FEF7E3F9C0F5807082B21249022094
:1005300000F0EAF80220FFF71FFE40F22555294699
:10054000204600F044F818B12946204600F01AF879
:1005500040F227752946204600F039F8002806D0D9
:1005600029462046BDE87040002200F050B870BD1A
:10057000004800409C000020443C00208A05C943FC
:100580000180704740F66A120A0A01219140C9436E
:1005900001807047002904D0818941F40051818194
:1005A0007047818921F4005181817047002A03D06E
:1005B000828A0A4382827047828A8A438282704793
:1005C0000246002012880A4200D00120704770B510
:1005D000002440F66A12C1F3421301F01F05012600
:1005E00006FA05F2012B0CD0022B0DD0838A1340A2
:1005F000090A8E40008830400BB100B1012420462A
:1006000070BD83891340F3E7038A1340F0E710B508
:1006100040F66A13C1F3421301F01F040121A14007
:10062000012B07D0022B07D014303AB102680A43DD
:10063000026010BD0C30F8E71030F6E702688A431C
:10064000026010BD30B585B004460D46208A4CF6D8
:10065000FF710840E98801432182A0894EF6F31119
:100660000840A9882A8911436A8902431143A1815C
:10067000A08A4FF6FF410840A9890143A18268463C
:10068000FFF7C4F91D48844201D1039800E00298A5
:10069000A189090408D500EBC00101EB001029680D
:1006A0004900B0FBF1F007E000EBC00101EB0010E6
:1006B00029688900B0FBF1F06422B0FBF2F1090176
:1006C0000B096FF018056B4300EB8300A3891D0431
:1006D0004FF0320307D503EBC000B0FBF2F000F09F
:1006E0000700084306E003EB0010B0FBF2F000F057
:1006F0000F000843208105B030BD000000380140E4
:10070000C1F308018180704730B40C46054951F8A7
:100710002030002B03D0204630BC1146184730BC97
:1007200070470000303A002010B50C46084A52F8D5
:100730002030002B09D0522206A10CA0FBF744FE6A
:100740000EA0FBF741FE204610BD42F82040FAE71C
:10075000303A00202E2E5C53595354454D5C55536E
:100760004152545C75736172742E63004C6F67451F
:1007700072723A2025732C25640000005561727452
:100780002043616C6C6261636B207265706561749B
:100790002072656721000000FEE7000010B50446E6
:1007A0000748FEF74FFE05230C2221460020FFF7E5
:1007B0000BFDBDE8104003490020FFF7B5BF000066
:1007C00022070020C907020810B50A46014605485D
:1007D000FEF742FE002804D0BDE8104002A0FEF75C
:1007E000C5BB10BD22070020735573625175657536
:1007F00065D2E7B3F6A3A100FEF76ABD2DE9F84F75
:1008000005462846FCF78FF800287BD02846FCF7E1
:100810008AF814301FFA80F8404600F0E7FB0746DC
:1008200000260024384B39A2414638460095FBF794
:10083000D7FD80B200F0010101EB5005FEF74CFC42
:100840003520FEF7DDFB10E00A20FEF793F80A2CB6
:1008500009D931A0FEF78AFBFEF73EFC3846BDE819
:10086000F84F00F0BFBB641CA4B20120FEF700FCEF
:100870000128E9D0DFF8B490DFF8B4A031E02020FF
:10088000FEF7BEFB701C81B2B85D08B940F02D00C8
:100890004A1C795C96B240EA0124200A01D144F452
:1008A0003454D9F80400C8F50061884207D3002009
:1008B000C9F80400B9F80800401CA9F80800D9F8E4
:1008C00004005044410501D1FEF7A0FBD9F8040013
:1008D00021465044FEF7E6FBD9F80400801CC9F815
:1008E00004006D1EADB2CAD2FFF78CF9FEF7D2FB41
:1008F00010A0D9F80410FDF7BDFB3846BDE8F84F4D
:1009000000F070BBBDE8F88FEF3F00202A25732070
:1009100025732A2000000000D0B4466C617368C3C0
:10092000A6B5C8B4FDB3ACCAB1A3A100280B002082
:1009300000F80708466C617368C6ABD2C6B3A4B6AC
:10094000C83A2523780000002DE9F04107460E46FD
:10095000002402F0010000EB52052120FFF7ACF863
:1009600001280AD0A82241A146A0FBF72DFD49A0ED
:10097000FBF72AFD0220BDE8F081FEF7ADFBA7F1F1
:100980000060B0F5002F01D278050BD0AE2237A160
:100990003CA0FBF719FD3FA0FBF716FDFEF77AFB25
:1009A0000220E8E7B5F5006F0BD9B4222FA135A0DE
:1009B000FBF70AFD37A0FBF707FDFEF76BFB0220F4
:1009C000D9E73520FEF71CFB3846FEF71FFB04284D
:1009D0001BD0BB2225A12BA0FBF7F6FC2DA0FBF71B
:1009E000F3FC12E00A20FDF7C5FF0A2C0BD9C22246
:1009F0001EA124A0FBF7E8FC26A0FBF7E5FCFEF710
:100A00006BFB0220B7E7641CA4B20120FEF730FBA9
:100A10000128E7D023E02020FEF7F2FA3078717841
:100A2000B61C40EA01213846FEF73CFB002410E0EA
:100A30000A20FDF79FFF1E2C09D9D3220BA111A07C
:100A4000FBF7C2FC13A0FBF7BFFC022093E7641C7A
:100A5000A4B22020FEF70CFB0128E9D1BF1C6D1EBB
:100A6000ADB2D8D2FEF716FB032084E72E2E5C53DE
:100A7000595354454D5C464C4153485C666C617318
:100A8000682E63004C6F674572723A2025732C25DF
:100A90006400000000000000490050EAC12018BFB7
:100AA00004204A0D18BF40F0010040F2FF72B2EB83
:100AB000515F08BF40F00200012808BF05207047C1
:100AC0002DE9F0414F1E00EBC7010446D1E90001BA
:100AD00015461E4637F006020DD02A46334602F070
:100AE00025FC7F1E04EBC703D3E9002302F074F951
:100AF00037F00602F1D1022F25D0042F13D0062F94
:100B000018BFBDE8F0812A46334602F00FFCD4E955
:100B10000A2302F061F92A46334602F007FCD4E9C1
:100B2000082302F059F92A46334602F0FFFBD4E9C4
:100B3000062302F051F92A46334602F0F7FBD4E9C6
:100B4000042302F049F92A46334602F0EFFBD4E9C8
:100B5000022302F041F92A46334602F0E7FBD4E9CA
:100B60000023BDE8F04102F037B90000002213462F
:100B70001046014902F0ECB90000F03F012202F0FA
:100B8000FFBD002213461046114602F0E1B930388D
:100B90000A2801D2012070470020704770470000EA
:100BA0000449C2B20B689A8009680A885206FCD5CB
:100BB0007047000064000020F0B503460025084699
:100BC00000260A2A01D00670F0BD002B1DD005DAE0
:100BD0004FF02D0200F8012BC3F1000342F2107216
:100BE0004FF00A0793FBF2F454EA050C06D004F127
:100BF000300500F8015B04FB1233012592FBF7F28C
:100C0000002AEFDC06700846F0BD30220270467004
:100C10000846F0BD2DE9F04DC84A002490B091423D
:100C200005DA21F00043934201D805D120B110B07C
:100C3000BDE8F04DFFF7A2BFB1F5801F1BDA53EA04
:100C4000000209D0002911DA0120FBF794FF10B04F
:100C5000BDE8F04DFFF795BF0220FBF78CFFFFF7D3
:100C600085FF10B081F00041BDE8F08D6FF03504D4
:100C7000362202F085FD04EB2152C1F31308B0497E
:100C8000A2F2FF33414401F4801282F07F6103EB52
:100C9000225281F04051009241EA08010022A94B02
:100CA00002F04EFC044608F10200A74EC0F3130008
:100CB0000D467E44032867D2D6E90023204602F081
:100CC0009FFA1ED10098002802BFD6E9000110B09B
:100CD000BDE8F08D02F0FFFA07460C469B4A9C4B9C
:100CE00002F024FB06460D469A4A9B4B38462146A5
:100CF00002F01CFB10B032462B46BDE8F04D02F06E
:100D00006BB84FF05532954B2046294602F00EFB4A
:100D10000022934B02F008FC06460F4622462B4663
:100D20001046194602F002FB32463B4602F0FEFA3C
:100D3000064600980F46F0B102F0CDFA80468A468A
:100D4000824A834B02F0F2FA32463B4602F0ECFB59
:100D500022462B4602F0F4FB05460C467D4A7E4BAC
:100D60004046514602F0E2FA10B02A462346BDE85A
:100D7000F04D02F0E5BB0B4610B032462046294646
:100D8000BDE8F04D02F0DCBB00224FF0804320466E
:100D900002F022F802460B462046294602F0D8F817
:100DA00006460F46009802F096FACDE90401324655
:100DB0003B461046394602F0B9FA0C9069480C9A45
:100DC0004044019009910B46104602F0AFFA82466A
:100DD000024665488B46C8F151080B4608F5D728EE
:100DE00003217844FFF76CFE52465B4602F09EFA00
:100DF0000A905E480D9152465B4604217844FFF705
:100E00005FFE099B0C9A02F091FA844601980D9BB3
:100E100040EA080860460A9A01F0DEFF834608911E
:100E2000B8F1000F4EDD4FF0FF322046294602F0A8
:100E3000A7FC22462B4602F079FA804600988A46A3
:100E400060B3DDE90401414A414B02F06FFA0991B8
:100E500000905A4640465146089B01F0BDFF32467D
:100E60003B4602F063FA099B009A01F0B5FF424647
:100E7000534602F059FB22462B4602F061FB044622
:100E80000D46DDE90401334A334B02F04FFA10B04E
:100E900022462B46BDE8F04D02F052BB5A46404672
:100EA000089B01F099FF32463B4602F03FFA42466A
:100EB000534602F039FB10B022462B46BDE8F04DF8
:100EC00002F032BB009840B3DDE904011F4A204B19
:100ED00002F02CFA80468A465A4620462946089B4C
:100EE00002F02EFB32463B4602F020FA42465346C1
:100EF00002F026FB22462B4602F022FB04460D465A
:100F0000DDE90401134A144B02F010FA10B0224636
:100F10002B46BDE8F04D02F013BB0B465A46204667
:100F2000294602F00DFB32463B4602F0FFF910B0B5
:100F300022462B46BDE8F04D02F0F6BA0000F07FE5
:100F4000645F09000000F03FFA2C0000763C793520
:100F5000EF39EA3D0000E0FE422EE63F5555D53F11
:100F60000000E03F86EBF9FF922B0000902B000081
:100F70001CB54FF4E0314FF00060FEF76BFCFFF75B
:100F80003BFC4FF44070FEF75BFC0E48FEF7BEF9E9
:100F90000D48FEF7A5F90D48FEF7ACF94FF4E13026
:100FA000FFF7FCFBFFF728FC09482021CDE90010E2
:100FB000CA00002307A10A4801F082FC01F0C0F832
:100FC00000201CBD2A06002010000020E7010020A0
:100FD0000400002073746172745F7461736B0000AD
:100FE000A5FD010801460020FEF71CBB70B50646B2
:100FF00031460020FEF722FB04460020FEF7D0FB1E
:1010000005464B2D08D9182215A11CA0FBF7DCF9C9
:1010100029461EA0FBF7D8F924B131462046FBF73C
:1010200020FD1BE020220EA114A0FBF7CDF92946DC
:101030001EA0FBF7C9F90020FEF746FB3146002051
:10104000FEF7FCFA04464CB9252205A10BA0FBF7DC
:10105000BBF923A0FBF7B8F9FEF74EFF204670BDA1
:101060002E2E5C53595354454D5C535953504F5297
:10107000545C737973706F72742E63004C6F6745A4
:1010800072723A2025732C25640000000D0AB6AF59
:10109000CCACC4DAB4E6D5BCD3C3D2D1B3ACB9FDC1
:1010A000A3BA25642525A3A10D0A00000D0AC4DA00
:1010B000B4E6D5BCD3C3A3BA256425252D2DB6AF80
:1010C000CCACC4DAB4E6D2E7B3F6A3A1B3F5CABC9C
:1010D000BBAFB6AFCCACC4DAB4E6BFD5BCE4A3A119
:1010E000000000002DE9F04104460F46174EF56858
:1010F0003068001D00F030FD38B9306890F82C10D1
:1011000001208840316981433161601C07D137B1CA
:101110003168BDE8F041091D0D4800F055BD2C4473
:1011200030684460AC4206D23168B06B091DBDE83E
:10113000F04100F031BD3168706B091D00F02CFDED
:10114000B06A844200D2B462BDE8F0814801002058
:10115000209B002070B5044600F042FD1D4DA8689C
:10116000401CA860286810B1686938B10CE02C6098
:10117000A868012808D100F099F905E02868E16A1B
:10118000C06A884200D82C60686A401C686260644B
:10119000E06A01212A698140114329610E4900EB6F
:1011A000800001EB8000211D00F00EFD00F054FDD9
:1011B000686900280CD02868E16AC06A884207D2B2
:1011C00006494FF080500860BFF34F8FBFF36F8F19
:1011D00070BD0000480100205098002004ED00E0A0
:1011E00010B500F0FDFC0E4C2068A0B90D4800F0D1
:1011F000C5FC0C48143000F0C1FC0A48E060143013
:10120000206100221021052001F07CF8206010B13F
:1012100005A100F0F7FDBDE8104000F01DBD000085
:1012200084010020349B0020546D725100000000A6
:1012300070B5124E124D1CE000F0CCFF306820B1AA
:10124000002401F09FFCA4B901E00124F9E700F0BB
:10125000C7FCF068C468201D00F07EFCA868401E32
:10126000A8606868401E686000F0F6FC204600F048
:1012700054F868680028DFD170BD00000C9B002086
:101280004801002030B40B46026C002A0CD0C16823
:101290001144C1604468A14201D30168C160C168C2
:1012A00030BC1846FBF75EBB30BC70472DE9F041FF
:1012B000044617460026A56B226C002A10D0C7B141
:1012C000E068FBF74FFBE168206C091AE1602268D7
:1012D000914202D26168081AE060022F16D017E02E
:1012E0002068A8B9606801F0A5FB06460020606090
:1012F0000EE0A068FBF736FB216CA0680844A060F4
:101300006168884204D32068A06001E005B16D1EC9
:101310006D1CA5633046BDE8F08110B50446206B16
:1013200000F0CEFC2046BDE8104000F0C9BC000033
:101330000749CA681168002904D00021016019B169
:10134000002070470121F9E7D0680068704700006D
:10135000840100204FF4B0410F48420706D0C01D61
:1013600020F007000C49411AC1F5B0410B4A10604A
:10137000002353600144083921F00701103A11603D
:101380004B600B600B1A43600160406890605060D6
:101390004FF00040D0607047104000203401002022
:1013A000074E4FF08054074DFFF742FF3068012889
:1013B000FAD92C60BFF34F8FBFF36F8FF4E70000B3
:1013C0005098002004ED00E070B51D46049C0029F3
:1013D0000BD02260E06321640121204601F094F8E3
:1013E00084F850500020A06470BD2460F2E7000033
:1013F0002DE9F047DDE908580A9C81460E4617465C
:101400009A46B900A522206BFBF723FB206B7F1EB9
:1014100000EB870020F00707780705D040F22E3256
:1014200019A11EA0FAF7D0FF00202218315C82F823
:101430003410315C11B1401C1028F6D3002684F81A
:101440004360202D00D31F25E562E5642665201D3D
:1014500000F09FFB04F1180000F09BFB2461C5F134
:101460002000A0616462666584F85860524649466F
:10147000384600F063FB2060B8F1000F01D0C8F8D7
:101480000040BDE8F08700002E2E5C467265655274
:10149000544F535C7461736B732E63004572726FAB
:1014A000723A25732C25640D0A00000070B50024E3
:1014B000114D04EB840005EB800000F05FFB641C21
:1014C000202CF6D30D4800F059FB0C48143000F0E6
:1014D00055FB0A48283000F051FB08483C3000F02A
:1014E0004DFB0648503000F049FB05480349416375
:1014F0001431816370BD000050980020D09A002004
:101500004801002030B5134900E011460A688242C4
:10151000FBD34B685C18844203D140681844486090
:1015200008460D6844682318AB420DD1094B103BA7
:101530001B689A4206D05268224442600A681268C8
:10154000026002E0036000E00260814200D00860B7
:1015500030BD00003401002070B5002441600061FE
:101560000C4D91420AD8D11A8269914201D30124CB
:101570000EE0011D286900F00FFB09E09A4203D23A
:10158000994201D3012403E0011DE86800F004FB47
:10159000204670BD8401002010B5044600F020FBF9
:1015A000A06B20B1002400F057FB204610BD0124A1
:1015B000F9E710B5044600F013FBA06BE16B88421D
:1015C00001D1012400E0002400F046FB204610BDBC
:1015D0002DE9F3410F460098846C0026002C05D1BC
:1015E00040F6CE1216A11BA0FAF7EEFEA06BE16B3F
:1015F000884205D340F6CF1211A116A0FAF7E4FEF7
:10160000A06BE16B88420CD294F945503A4669468A
:101610002046FFF74BFE0646681C05D06D1C84F87B
:1016200045503046BDE8FC81606A0028F9D004F1DD
:10163000240001F059FA0028F3D00126F1E7000058
:101640002E2E5C4672656552544F535C71756575FC
:10165000652E63004572726F723A25732C25640DF6
:101660000A000000F8B505460E461348C068C06879
:10167000C468201D00F070FAE069012816D1A06945
:101680002B46411932462046FFF766FF70B1002015
:101690000346014600902A46204601F023FB28B964
:1016A0004FF4027205A10BA0FAF78EFE616A01B039
:1016B0002046BDE8F0400847840100202E2E5C46FD
:1016C00072656552544F535C74696D6572732E6315
:1016D000000000004572726F723A25732C25640D6C
:1016E0000A00000070B586B02F4E53E00298002823
:1016F00003DADDE90320059990470298002849DBC9
:10170000049C606910B1201D00F026FA01A800F0C9
:10171000A9F8054602980A283CD2DFE800F0050542
:10172000053B273805053B270398A169034601447B
:101730002A462046FFF710FF00282BD0616A20467A
:101740008847E069012825D1002000900398A1690D
:10175000002342181946204601F0C4FAD0B940F2DD
:10176000213212A117A0FAF72FFE13E00398A0610F
:1017700028B94FF44E720DA112A0FAF725FEA06908
:101780002B4641192A462046FFF7E6FE02E0204696
:1017900000F096FA00231A4602A9306800F0E4FD32
:1017A0000028A3D106B070BD840100202E2E5C4617
:1017B00072656552544F535C74696D6572732E6324
:1017C000000000004572726F723A25732C25640D7B
:1017D0000A000000F8B506460D4600F0FBFC68461E
:1017E00000F040F80446009810B101F0CBF9F8BDC4
:1017F00045B9A64206D801F0C5F921463046FFF7A3
:1018000031FFF8BD0C481DB10169096891B100258F
:10181000311B2A46006800F007FB01F0B3F90028ED
:10182000EFD106494FF080500860BFF34F8FBFF3F0
:101830006F8FF8BD0125EBE78401002004ED00E087
:101840000748416B0968002905D0416BC968C96820
:101850004968816270474FF0FF3181627047000034
:101860004801002070B5054601F068F80446074EAF
:10187000B068844204D200F00BF80120286001E037
:1018800000202860B460204670BD00008401002064
:10189000F8B5184E25E0C0680568C468201D00F042
:1018A0005BF9616A20468847E069012819D1A0697F
:1018B0002844A84206D960602461211DF06800F028
:1018C0006BF90EE000200346014600902A462046B0
:1018D00001F008FA28B940F2923207A10CA0FAF7F9
:1018E00073FDF06801680029D5D1F0683169F160B5
:1018F0003061F8BD840100202E2E5C467265655271
:10190000544F535C74696D6572732E630000000060
:101910004572726F723A25732C25640D0A0000001F
:1019200008484068401C04D0F52207A111A0FAF72E
:101930004BFD502080F31188BFF34F8FBFF36F8FA3
:10194000FEE700003C0100202E2E5C4672656552C9
:10195000544F535C706F727461626C655C52564494
:10196000535C41524D5F434D335C706F72742E6314
:10197000000000004572726F723A25732C25640DC9
:101980000A00000008B56846FFF7D2FC0099FFF78F
:1019900021FFFFF7A7FEF6E72DE9F041044600F02E
:1019A0001FF994F9455004F1240613E0A06C38B1F6
:1019B00000212046FFF70CFE50B100F0F7FA07E0D7
:1019C000606A48B1304601F08FF808B100F0EEFAD5
:1019D0006D1E6DB2002DE9DC4FF0FF3684F84560D6
:1019E00000F03AF900F0FCF894F9445004F11007C3
:1019F00009E0206948B1384601F076F808B100F0F6
:101A0000D5FA6D1E6DB2002DF3DC84F84460BDE89C
:101A1000F04100F021B900002DE9F0410546002613
:101A200000F0D8FB304F386808B9FFF793FCF8682E
:101A300005424BD175B1083568070BD005F007009A
:101A4000C0F108000544680704D0C02227A131A0D6
:101A5000FAF7BAFC002D39D07868854236D8224989
:101A600010310846046801E0214604466068A84237
:101A700002D220680028F7D13868844226D00E6848
:101A80000836206808606068401B102811D904EBF4
:101A900005085FEA487004D0ED2214A11DA0FAF7F2
:101AA00093FC6068401BC8F8040065604046FFF77F
:101AB00029FD61687868401A7860BA68904200D25F
:101AC000B860F868014361600020206001F05AF8B6
:101AD000700705D040F22D1204A10EA0FAF774FC95
:101AE0003046BDE8F0810000240100202E2E5C4627
:101AF00072656552544F535C706F727461626C65AD
:101B00005C4D656D4D616E675C686561705F342E1C
:101B1000630000004572726F723A25732C25640DC4
:101B20000A00000004490868002803D00868026D14
:101B3000521C0265086870474801002020384FF0A9
:101B40008073C36121F0010181610249416140F864
:101B500020297047211902080169D0E901329A60F1
:101B6000D0E901235A604A68824201D182684A6002
:101B7000002202610868401E0860704700F10801F9
:101B800041604FF0FF328260C1600161002101605D
:101B9000704700210161704730B50C68621C02D0AB
:101BA00000F1080202E0026904E01A4653681D6869
:101BB000A542FAD953684B6099608A605160086108
:101BC0000168491C016030BD42684A6093688B60BF
:101BD00093685960916008610168491C0160704711
:101BE000502080F31188BFF34F8FBFF36F8F0949E7
:101BF0004868401C486001280AD10748006810F076
:101C0000FF0F05D04FF4C07204A10FA0FAF7DCBBA0
:101C1000704700003C01002004ED00E02E2E5C46E1
:101C200072656552544F535C706F727461626C657B
:101C30005C525644535C41524D5F434D335C706F70
:101C400072742E63000000004572726F723A257341
:101C50002C25640D0A00000010B5094C60680028AE
:101C600005D140F2871207A111A0FAF7ADFB606819
:101C7000401E6060002801D180F3118810BD000073
:101C80003C0100202E2E5C4672656552544F535C19
:101C9000706F727461626C655C525644535C415261
:101CA0004D5F434D335C706F72742E630000000013
:101CB0004572726F723A25732C25640D0A0000007C
:101CC00070B500282AD008380446154D6068E968C8
:101CD000084205D14FF4A27212A11CA0FAF774FBBE
:101CE000206828B140F245120EA118A0FAF76CFB4B
:101CF0006068E968084211D02268002A0ED1884342
:101D0000606000F067FA60686968084468602046AF
:101D1000FFF7F8FBBDE8704000F034BF70BD000075
:101D2000240100202E2E5C4672656552544F535C90
:101D3000706F727461626C655C4D656D4D616E674C
:101D40005C686561705F342E630000004572726FDD
:101D5000723A25732C25640D0A00000005486421A1
:101D60000068B0FBF1F14FF0E020491E416107210E
:101D7000016170471001002010B5FAF7E5FA104C28
:101D800010280CD300F1E02090F8F003217888426D
:101D900005D240F2AE220BA115A0FAF715FB1848A8
:101DA0000068A16800F4E060884207D9BDE81040EF
:101DB00040F2BE2203A10EA0FAF706BB10BD000040
:101DC0003C0100202E2E5C4672656552544F535CD8
:101DD000706F727461626C655C525644535C415220
:101DE0004D5F434D335C706F72742E6300000000D2
:101DF0004572726F723A25732C25640D0A0000003B
:101E00000CED00E010B50022064B53F832401CB137
:101E1000521C082AF9D310BD43F8321003EBC2015B
:101E2000486010BD1098002070B504460D46164657
:101E3000FFF7D6FE94F944304FF000005B1C01D14F
:101E400084F8440094F94510491C01D184F84500F8
:101E5000FFF702FFA06B28B93246294604F124009F
:101E600000F0D6F82046BDE87040FFF795BD0000B1
:101E700010B504460020002C10D00E48006B28B18D
:101E800040F2D2420CA111A0FAF79EFA00F0A2F99A
:101E900000212046FFF726F900F074FE002807D144
:101EA0000E494FF080500860BFF34F8FBFF36F8F24
:101EB00010BD0000480100202E2E5C467265655260
:101EC000544F535C7461736B732E63004572726F71
:101ED000723A25732C25640D0A00000004ED00E021
:101EE00070B50446FFF77CFE234D04B92C68201D15
:101EF000FFF732FE58B9E06A204A00EB800152F841
:101F0000211021B901218140286988432861A06AF4
:101F100018B104F11800FFF71FFE686A401C6862E0
:101F20002868844207D1211D1548FFF74DFE6868D7
:101F3000401C686007E0A868401EA8602046FFF7C4
:101F4000ECF9FFF77DFCFFF787FE6869002812D0E7
:101F5000286884420FD1286B28B14FF48D6209A103
:101F60000DA0FAF731FA10494FF080500860BFF326
:101F70004F8FBFF36F8F70BD480100205098002035
:101F80000C9B00202E2E5C4672656552544F535CAC
:101F90007461736B732E63004572726F723A2573AE
:101FA0002C25640D0A00000004ED00E00149012029
:101FB000C86170474801002070B504460D46002CEA
:101FC00005D140F60F3208A10CA0FAF7FDF90F4831
:101FD000016820461831FFF7DFFD2846BDE8704054
:101FE0000121FFF77FB800002E2E5C467265655216
:101FF000544F535C7461736B732E63004572726F40
:10200000723A25732C25640D0A0000004801002057
:1020100070B506460D461446002E05D140F63A32FC
:1020200009A10EA0FAF7D0F910480168304618311E
:10203000FFF7CAFD0CB14FF0FF3521462846BDE839
:102040007040FFF74FB800002E2E5C467265655257
:10205000544F535C7461736B732E63004572726FDF
:10206000723A25732C25640D0A00000048010020F7
:1020700070B50446002839D01D4DE06A2968C96A48
:10208000884233D2A069002804DB2868C06AC0F106
:102090002000A061E06A174E00EB8000616906EB4A
:1020A000800081421FD1201DFFF756FD012150B94C
:1020B000E06A00EB800256F8222022B92A6901FA70
:1020C00000F082432A612868C06AE0622A69814080
:1020D0001143296100EB800006EB8000211DBDE863
:1020E0007040FFF771BD2868C06AE06270BD0000F3
:1020F000480100205098002010B50446002C05D15E
:1021000040F6CA3204A109A0FAF75EF90B48016A49
:102110002160C068606010BD2E2E5C4672656552FD
:10212000544F535C7461736B732E63004572726F0E
:10213000723A25732C25640D0A0000004801002026
:102140001CB517480024CDE900402346822215A182
:10215000164800F0B5FB012801D100F089FD0128E7
:102160000AD0401C1BD102B04FF4F162BDE8104010
:102170000FA114A0FAF728B9502080F31188BFF3FB
:102180004F8FBFF36F8F06484FF0FF312C388162BD
:1021900001214161C460BDE81C4000F063B81CBD72
:1021A0007401002049444C4500000000A1130208BE
:1021B0002E2E5C4672656552544F535C7461736B8E
:1021C000732E63004572726F723A25732C25640D6D
:1021D0000A0000000248016B491C016370470000BF
:1021E0004801002070B5144D286B002802D0012052
:1021F000E86170BD0020E8612869B0FA80F0C0F1A4
:102200001F000E4E00EB800456F8240028B940F65B
:10221000FF220BA10FA0FAF7D7F806EB8400416864
:102220004968416000F10802914201D1496841606A
:102230004068C068286070BD4801002050980020A8
:102240002E2E5C4672656552544F535C7461736BFD
:10225000732E63004572726F723A25732C25640DDC
:102260000A0000001CB5194908780190FF20087089
:10227000087800909DF80000154A00F0500010709A
:102280000720906006E09068401E90609DF8000076
:10229000400000909DF800000006F4D4107A00027F
:1022A00000F4E0609060019808700A48016841F409
:1022B00070010160016841F070410160FFF74EFD5F
:1022C00000205060FAF70AF800201CBD00E400E08E
:1022D0003C01002020ED00E010B5502080F3118873
:1022E000BFF34F8FBFF36F8F00F02EFB18B104497F
:1022F0004FF080500860002080F3118810BD00006E
:1023000004ED00E0F8B505460E461746002D05D150
:102310004FF4C4720BA110A0FAF756F886B105FB72
:1023200006F05430FFF778FB04463CB104F1540248
:102330003B46314628460094FFF746F82046F8BD54
:102340000020EEE72E2E5C4672656552544F535CBA
:1023500071756575652E63004572726F723A2573EB
:102360002C25640D0A0000002DE9FF4F83B00446C0
:102370008A469B460026002C05D140F2DC4258A13B
:102380005CA0FAF721F8BAF1000F07D1206C28B150
:1023900040F2DD4252A157A0FAF716F800F0C0FA59
:1023A00038B9059828B14FF49C624DA151A0FAF7B5
:1023B0000BF84FF000094FF08057DFF84881FFF726
:1023C0000FFCA56B95B3E66851462046FEF75AFF11
:1023D000BBF1000F13D0E660606A50B104F1240035
:1023E00000F082FB28B1C8F80070BFF34F8FBFF335
:1023F0006F8FFFF731FC012007B0BDE8F08F6D1E35
:10240000A563206810B9FFF78DFB60602069002884
:10241000EFD004F1100000F067FB0028E9D0C8F805
:102420000070BFF34F8FBFF36F8FE2E7FFE70598B0
:1024300008B126B107E0FFF70FFC0020DCE701A898
:10244000FFF75AFE0126FFF707FCFFF7C3FEFFF771
:10245000C7FB94F94400401C01D184F8449094F9DE
:102460004500401C01D184F84590FFF7F5FB05A914
:1024700001A800F0DDF958B12046FFF78DFA00F011
:1024800081FB2046FFF788F8002898D00020B3E7AA
:102490002046FFF781F8E0B1206830B9FFF7A0FBD4
:1024A0006068FFF7E5FDFFF7D7FB04F1240005990D
:1024B000FFF782FD2046FFF76FFA00F063FB00286C
:1024C0007FF47DAFC8F80070BFF34F8FBFF36F8FFD
:1024D00075E72046FFF760FA00F054FB6FE7000055
:1024E0002E2E5C4672656552544F535C717565754E
:1024F000652E63004572726F723A25732C25640D48
:102500000A00000004ED00E070B504460D46002C02
:1025100005D140F21B121DA121A0F9F755FFFFF7CD
:102520005FFBD4E90F20216802FB001161600021EC
:10253000A1632168A160E06B2268216C401E00FB52
:102540000121E1604FF0FF3084F8440084F8450039
:1025500004F110004DB1FFF711FB04F12400FFF767
:102560000DFBFFF779FB012070BD21690029F8D030
:1025700000F0BAFA0028F4D00D494FF080500860FE
:10258000BFF34F8FBFF36F8FEBE700002E2E5C463B
:1025900072656552544F535C71756575652E6300A5
:1025A0004572726F723A25732C25640D0A00000083
:1025B00004ED00E02DE9FF4782B004468A469846C4
:1025C0000025002C05D140F2D92254A158A0F9F7DA
:1025D000FBFEBAF1000F07D1206C28B140F2DA22DD
:1025E0004EA153A0F9F7F0FEB8F1020F08D1E06B4D
:1025F000012805D040F2DB2248A14DA0F9F7E4FE06
:1026000000F08EF938B9049828B140F2DE2243A1D7
:1026100047A0F9F7D9FE4FF000094FF08056484F18
:10262000FFF7DEFAA06BE16B884206D3B8F1020F28
:1026300003D0049860B37DB333E042465146204650
:10264000FEF734FEA16C51B141462046FEF7C0FFB3
:10265000C0B13E60BFF34F8FBFF36F8F12E0616A6E
:1026600051B104F1240000F03FFA58B13E60BFF3CD
:102670004F8FBFF36F8F05E020B13E60BFF34F8FE8
:10268000BFF36F8FFFF7E8FA012006B0BDE8F087CF
:10269000FFF7E2FA0020F8E7FFE76846FFF72CFDB6
:1026A0000125FFF7D9FAFFF795FDFFF799FA94F99D
:1026B0004400401C01D184F8449094F94500401C2A
:1026C00001D184F84590FFF7C7FA04A9684600F0E5
:1026D000AFF830B12046FFF75FF900F053FA002061
:1026E000D3E72046FEF765FF88B104F11000049996
:1026F000FFF762FC2046FFF74FF900F043FA00288D
:102700008ED13E60BFF34F8FBFF36F8F88E72046B7
:10271000FFF742F900F036FA82E700002E2E5C4601
:1027200072656552544F535C71756575652E630013
:102730004572726F723A25732C25640D0A000000F1
:1027400004ED00E02DE9F047044689461546984619
:10275000002C05D140F29F322CA131A0F9F734FEB4
:10276000B9F1000F07D1206C28B14FF4687227A18E
:102770002BA0F9F729FEB8F1020F08D1E06B012870
:1027800005D040F2A13221A125A0F9F71DFEFFF7E7
:10279000F3FA5020EFF3118780F31188BFF34F8FC6
:1027A000BFF36F8FA06BE16B884207D3B8F1020FC4
:1027B00004D0002087F31188BDE8F08794F94560C4
:1027C000424649462046FEF771FD701C04D0761C37
:1027D00084F845600120EDE7A06C012648B1414630
:1027E0002046FEF7F5FE0028F4D0002DF2D02E6032
:1027F000F0E7606A0028EDD004F1240000F074F9DD
:102800000028E7D0002DE5D02E60E3E72E2E5C46B1
:1028100072656552544F535C71756575652E630022
:102820004572726F723A25732C25640D0A00000000
:1028300070B504460D46002C05D140F6D43216A1E1
:102840001AA0F9F7C1FD2DB940F6D53212A117A093
:10285000F9F7BAFDFFF7C4F9184AD06829684B1C8C
:1028600008D02368126A934206D06268824203D875
:1028700001240DE000240BE06268801A884206D231
:10288000081A28602046FFF737FC002400E00124E6
:10289000FFF7E2F9204670BD2E2E5C467265655248
:1028A000544F535C7461736B732E63004572726F87
:1028B000723A25732C25640D0A000000480100209F
:1028C0002DE9FF5F8146DDE90E788A4616469B4674
:1028D000B000FFF7A1F8054628000AD05C20FFF7FA
:1028E0009BF804460CB1256304E02846FFF7E8F99D
:1028F00000E000248CB10020CDE90240CDE9007851
:102900005B46324651464846FEF772FD2046FEF7CA
:1029100021FC012004B0BDE8F09F4FF0FF30F9E743
:1029200005484169002903D0006B18B100207047A9
:102930000120704702207047480100200148C0680C
:1029400070470000480100202DE9F04100262E4F7D
:10295000386B002808D0B869401CB861F86900B12C
:1029600001263046BDE8F081FD686D1CFD608DB923
:10297000786B006828B140F6DE1224A128A0F9F790
:1029800023FD786BB96B7963B863386A401C386291
:10299000FEF756FFB86ADFF8988085420DD3786B52
:1029A000006838B1786BC068C468606885420ED230
:1029B000B86202E04FF0FF30B8623868C06A00EBDE
:1029C000800058F820000128C8D90126C6E7201D3C
:1029D000FFF7C2F8A06A18B104F11800FFF7BCF8BD
:1029E000E06A01213A6981401143396100EB8000BE
:1029F00008EB8000211DFFF7E7F8E06A3968C96A33
:102A00008842CCD30126CAE7480100202E2E5C461E
:102A100072656552544F535C7461736B732E63001F
:102A20004572726F723A25732C25640D0A000000FE
:102A30005098002070B50446002600283CD01F4D59
:102A40002868844205D04FF46D621DA121A0F9F7DA
:102A5000BBFC206D28B940F6D26219A11DA0F9F780
:102A6000B3FC206D401E2065E26CE16A914223D0E8
:102A700010BB201DFFF770F81A4A012150B9E06A17
:102A800000EB800352F8233023B92B6901FA00F0E0
:102A900083432B61E06CE062C0F12000A061E06A3A
:102AA0002B6981401943296100EB800002EB800013
:102AB000211DFFF789F80126304670BD480100202E
:102AC0002E2E5C4672656552544F535C7461736B75
:102AD000732E63004572726F723A25732C25640D54
:102AE0000A000000509800202DE9F041C068C46839
:102AF000002C05D140F66A3216A11BA0F9F764FC40
:102B000004F118000746FFF727F81B4D2A6B012632
:102B100062B139461948FFF757F8E06A2968C96A6F
:102B2000884215D90120EE61BDE8F081201DFFF734
:102B300013F8E06A2A6906FA00F111432961104985
:102B400000EB800001EB8000211DFFF73DF8E4E77A
:102B50000020E9E72E2E5C4672656552544F535CA7
:102B60007461736B732E63004572726F723A2573D2
:102B70002C25640D0A00000048010020F89A00206E
:102B8000509800202DE9F041002400272B4D286BA0
:102B9000002805D140F2EC7229A12EA0F9F714FC0F
:102BA000FFF71EF8286B401E2863286BF0BBA8684F
:102BB000E0B3DFF8B08001261DE0D8F80C00C4684F
:102BC00004F11800FEF7C8FF201DFEF7C5FFE06AFC
:102BD0002A6906FA00F111432961234900EB8000BC
:102BE00001EB8000211DFEF7EFFFE06A2968C96A4A
:102BF000884200D3EE61D8F800000028DDD10CB186
:102C0000FEF71EFEAC6944B1FFF79EFE00B1EE6117
:102C1000641E002CF8D10020A861E86930B10127BA
:102C2000124938070860BFF34F8F00E001E0BFF39F
:102C30006F8FFFF711F83846BDE8F081480100209A
:102C40002E2E5C4672656552544F535C7461736BF3
:102C5000732E63004572726F723A25732C25640DD2
:102C60000A000000F89A00205098002004ED00E0CF
:102C70001CB50024FEF7B4FA0C48006860B10B489C
:102C80001F21001DCDE9001000234FF4827208A11E
:102C90000948FFF715FE04462CB940F2331207A18C
:102CA0000CA0F9F791FB20461CBD00008401002018
:102CB000546D722053766300851902082E2E5C46EF
:102CC00072656552544F535C74696D6572732E63FF
:102CD000000000004572726F723A25732C25640D56
:102CE0000A0000002DE9FF47DDF830A005460E463A
:102CF000904699460027002D05D14FF4D37215A1B7
:102D00001AA0F9F761FB1D4C2068F8B10096CDF8C8
:102D100004800295062E13DAFFF702FE022807D080
:102D200000231A4669462068FFF744FC07460DE079
:102D30000023524669462068FFF73CFC074605E041
:102D400000234A466946FFF7FDFC074604B03846B3
:102D5000BDE8F0872E2E5C4672656552544F535C79
:102D600074696D6572732E63000000004572726FA6
:102D7000723A25732C25640D0A000000840100209E
:102D800010B500290AD00878002807D005487844F3
:102D9000FAF768FD002801D0002010BD02487844F1
:102DA00010BD00009A0D0000920D000010B5002922
:102DB0000AD00878002807D005487844FAF752FD71
:102DC000002801D0002010BD0248784410BD00004A
:102DD0007E0E0000760E000010B591EA030F48BF8A
:102DE00083F0004300F1B483841A71EB030C05D225
:102DF000121943EB0C03001B61EB0C01DFF824E11B
:102E00004FEA1154A4EB135C1EEA430F18BF9EEA6D
:102E1000445F73D023EA0E03DCF1200E21EA045153
:102E200043F4801332D322FA0CFE10EB0E0023FA87
:102E30000CFE41EB0E01CCF1200E03FA0EFE10EB5E
:102E40000E0051F10001B1F5801FCCF1200E32D2FD
:102E500001EB045112FA0EF2BDE8104058BF704762
:102E6000401C38BF5FEA420218BF7047002814BFF9
:102E700020F0010041F100014FEA410313F5001F6A
:102E800038BF7047A1F1C04100F048BB012A43EBB5
:102E90000302ACF1200CDCF11F0E32BF4FF0000E2C
:102EA00023FA0CF310EB030041EB0451B4EB115F78
:102EB000D0D0A1EB045101F5801149085FEA300040
:102EC00001EB04510ED350F1000038BF12FA0EFE90
:102ED00008D1BDE81040C9E7401C38BF5FEA420294
:102EE000CAD1C3E7BDE810404FEA410313F5001F04
:102EF00038BF7047A1F1C04100F010BB9EEA445FAB
:102F000008D011EA5E0FBDE8104004BF01F0004197
:102F100000207047BDE8104070B500F0B1FA00BF66
:102F200064FBBE3E0000E0FF02494FF0000000F0ED
:102F3000F5BB00BF0000F87F491058BFC1F1404108
:102F40005B1058BFC3F140438B42EFF300807047E2
:102F50002DE9C04130B4DFF8A0C23CEA111418BF1B
:102F60003CEA131400F0EC8081EA03051CEA11141A
:102F700044EAD57418BF1CEA131500F0C780A4EB0F
:102F800005044FF0004545EAC12145EAC32341EA63
:102F9000505143EA525304F17F74994204F50034CE
:102FA0004FEAC0204FEAC22208BF904200F09C8046
:102FB0004FEA13650FF24016765D4FEA134506FBA4
:102FC00005F7C7F1807706FB07F74FEAD737A7FB6E
:102FD00003687642C8F58038A7FB06CE38BFA8F153
:102FE000010807FB08E64FF0000EA6FB028CE6FB8B
:102FF00003CEDCF1000CCEF1004E38BFAEF1010E75
:10300000A6FB0C584FF000074FF00005E6FB0E87BB
:10301000A1FB08C6A0FB07CE16EB0E0645F1000586
:10302000E1FB076515F1E04E7EBFA4F580345FEA51
:1030300046066D4116F1800745F100054FEA172756
:103040004FEA066647EA0567A6F1DE46B6F1805FFD
:103050004FEA15251FD9384624F0010C05EBC47141
:10306000BCF1FE6F01EB0C1102D8F0BCBDE8008191
:1030700024425CBF01F5801E9EEAC47F02D4F0BCEE
:10308000BDE80081244238D4F0BCA1F1C041BDE8C4
:10309000004100F043BA4FEAD22242EA43524FEADB
:1030A000D323A7FB02864FEAD02040EA415007FB1A
:1030B00003661EEA0E0F4FEAD12105FB026658BFD8
:1030C000A6EB0056B6EB00564FEA520E4EEAC37E10
:1030D00018EB0E0E56EB530EBDD518EB02085E41F1
:1030E0007F1C55F10005B6E74FF480154FF000073F
:1030F0004FF000064FF00008ADE7F0BC4FF00000C5
:1031000001F1C04101F00041BDE8008111EA0C1F4E
:103110000CEA131500D00CE013EA0C1F00F0258018
:103120004FF00000F0BC81EA030101F00041BDE86E
:103130000081F0BCBDE8004181EA030100F0EEB976
:10314000F0BCBDE8004170B500F09AF9097EFC3E84
:1031500000F007B881EA03014FF0000001F00041E0
:10316000704781EA030100F0D9B9F0BCBDE8004125
:103170004FF0000021497047FFFDFBF9F7F5F4F22D
:10318000F0EEEDEBE9E8E6E4E3E1E0DEDDDBDAD802
:10319000D7D5D4D3D1D0CFCDCCCBCAC8C7C6C5C460
:1031A000C2C1C0BFBEBDBCBBBAB9B8B7B6B5B4B377
:1031B000B2B1B0AFAEADACABAAA9A8A8A7A6A5A462
:1031C000A3A3A2A1A09F9F9E9D9C9C9B9A99999826
:1031D0009797969595949393929191908F8F8E8EC9
:1031E0008D8C8C8B8B8A8989888887878685858456
:1031F00084838382828181800000FF070000F87F42
:1032000051EA030C17D41CF5801F58BFBCF5801F72
:1032100000F10680994218BF704708BF904270477E
:1032200007D711F5801F58BF13F5801F19D4994295
:103230007047894270471CF5801F08D5BCF5801F78
:10324000F7D58B4218BF704708BF824270474FF4D2
:10325000001C1CEB410F38BF1CEB430F01D28B420B
:10326000704770B500F00CF9922449004FF00051FE
:103270004FF08053FFF760BE4FEA41034FEA5353CC
:10328000A3F58063D3F11E03C8BFD3F1210C0CDD7D
:103290004FF0004242EAC12242EA505232FA03FCA5
:1032A0008CEAE17CACEBE1707047102BC4BF0020CE
:1032B000704703F5787CBCF1FF3F04D06FF000420B
:1032C00082EA2100704770B500F0DAF84992248054
:1032D00000207047F2E710F0004248BF4042B0FAC9
:1032E00080F310FA03F10AD0C3F11D0303F58063E4
:1032F0004FEA415002EB035202EBD12170474FF0ED
:1033000000007047B0FA80F310FA03F10AD0C3F15D
:103310001D0303F580634FEA41504FEA035202EB6D
:10332000D12170474FF0000070470000DFF848C11E
:1033300070B51CEA111E1EBF1CEA13159EEA0C0F85
:1033400095EA0C0F00F06F8081EA030423EA4C1326
:103350004EEAD47E21EA4C1141F4801143F48013EB
:10336000AE44A1FB024CA0FB0365AEF17F7E361993
:1033700055EB0C05A1FB034C4CF10003A0FB021C18
:1033800016EB0C06654153F10003094218BF46F0E5
:10339000010613F4007F0BD14FEA03314FEA0530E9
:1033A000340341EA155140EA16506FF003020AE077
:1033B0004FEAC3214FEAC520F40241EA555140EAE1
:1033C00056506FF0020202EB2E4201EB025585EAE5
:1033D000CE710AD05FEA440C18BF24F0004450F1CB
:1033E000000041F1000120EAD47040F2FE7C624509
:1033F00000D270BDA84214BF4FF080444FF040444B
:10340000002E08BF0024BEF1806FA8BFA1F1C0410B
:10341000BDE8704080F282804FF0000001F1C041B1
:1034200001F0004170479EEA0C0F0CEA131518BF1B
:1034300095EA0C0F06D04FF0000081EA030E0EF063
:10344000004170BD00F01CF88900013E00F007B893
:1034500000F009B84FEA430C5FEA5C5C08D081EAEF
:10346000030100F05BB84FEA410C5FEA5C5CF6D107
:103470004FF00000014970470000FF070000F87F8F
:103480000EF1020E2EF0030E5EF8046B364205D4E8
:10349000012A43EB030515F5001F12D8012841EB63
:1034A000010C1CF5001F0CD80ED14FEAD17C15F58C
:1034B000001F0CEB4C0C0CF1020C08BF4CEBD37C46
:1034C00004E04FF0080C01E04FEAD37C0CEB4C0514
:1034D00026FA05F606F00706B6F1040C06D20EEB46
:1034E000860CBDE870404CF0010C6047DFE80CF042
:1034F000090B02024FF000414FF00000A1F500213E
:1035000070BD19461046012851EB010418BFD4F5CF
:10351000001484BF002001F0004170BD0808A0F530
:1035200000114FEA3101704791EA030F10B581F0A5
:1035300000413FF559AC83F0004300F009B80000AA
:1035400010B591EA030F48BF83F000433FF54CAC40
:10355000841A71EB030C07D212198CF0004C43EB68
:103560000C03001B61EB0C01DFF8A4E14FEA1154DE
:10357000A4EB135C1EEA430F18BF9EEA445F00F001
:10358000B08023EA6E03524221EA0451C3EB6E037A
:1035900038BF5B1EDCF1200E25D322FA0CFE10EBA7
:1035A0000E0043FA0CFE41EB0E01CCF1200E03FAA3
:1035B0000EFE10EB0E0051F10001CCF1200E29D4CB
:1035C00012FA0EF201EB0451BDE8104058BF7047EB
:1035D000401C1CBFB2F1004F704700280CBF491CB3
:1035E00020F00100704712EB020E43EB030218BFFC
:1035F0004FF0010E4EEA4202ACF1200CDCF11E0E3F
:1036000054D943FA0CFE10EB0E0051F1FF31CCF10E
:103610001E0ED5D50EF1010E12FA0EFE404141EB01
:10362000010101EB445C5FEA5C5C10D910EBDE70D9
:1036300001EB045138BFBEF1004FBDE8104018BF88
:10364000704700280CBF491C20F00100704730D2A1
:103650004FEAD42C11F5001124F400641BD0B1FA08
:1036600081F20B3AA41AA41ED2F12003914030FA41
:1036700003F31943904001EBCC71002C01EB045192
:10368000BDE81040A8BF704701F1C0414FF00000F5
:1036900001F000417047B0FA80F310FA03F100D155
:1036A00010BDE41A173C4805C90AE4E701EB0451D0
:1036B00010BD491001EB0451BDE810404FEA300045
:1036C00002E04FF0000170474A0008BF0042F8D006
:1036D000B2F5001F28BF704701F000414FF0000015
:1036E00070479EEA445F07D011EA5E0FBDE81040C4
:1036F00004BF002100207047BDE8104070B5FFF7FF
:10370000BFFE00BF40DFF63E83F000411046704729
:103710000000E0FFF9F767BBF9F7E4BD0CF00F0319
:10372000092B08BF082000F059800A2B0BD0082B6A
:1037300018BF704708BF1CF0400F0AD04FF00000C0
:103740004FF0000170471CF0400F18BF4FF00040D1
:1037500070471CF0100F08D020F0704300F07F423B
:1037600042EAD3014FEA4370704700F0604021F015
:103770007F4242EA000201F07F4040EA72707047E7
:103780004FF0FF0C4CF4E06C1CEA11531CBF9CEA98
:10379000030C9445C2BFDA4201EB02517047002B83
:1037A0000DD0BCF1000F0FD0002A01F00041A4BFE2
:1037B00041F0E04141F07F614FF00000704701F0BF
:1037C00000414FF00000704750EA01334FF09B0C6E
:1037D00018BF4CF0806C7FF4A7AB70471CF4801FBF
:1037E00011D01CF4E02F03D06FEACC3149007047B0
:1037F0004FF04050EFF3008222F0704242EA0002A4
:1038000082F3008870474FF00000704760010000AD
:10381000010000002000000020000000002C00003B
:10382000200000000306010B0405020925262734A9
:10383000350000010001000100010000004000000F
:10384000000002000000040000000800000010005A
:10385000443A0020443B0020443C0020443D0020EA
:103860000B0000000C0000000D0000000E00000026
:103870000F000000100000001100000038000000E0
:10388000390000003A0000003B0000003B0000004F
:103890000001020304050600040000000800000007
:1038A0001000000020000000400000008000000028
:1038B00000010000010002000400080010002000C8
:1038C00040008000000100020004000800100020F9
:1038D00000400080000102030405060708090A0BE6
:1038E0000C0D0E0F0100000002000000040000009B
:1038F0000800000010000000200000004000000050
:103900008000000000010000000200000004000030
:10391000000800000010000000200000004000002F
:1039200000800000060708090A171717171728282C
:103930002828282800000000000000003031323321
:1039400034353637383941424344454640305800D3
:103950003031323334353637383961626364656605
:103960004030780004000008000000000000000261
:10397000000100001000000004FA97999999D93FBE
:10398000AF788E1DC571CC3F9FC678D0099AC33FD2
:10399000935555555555E53F599322942449D23FA7
:1039A000DE03CB966446C73F44523EDF12F1C23F6E
:1039B000000000000000000030313233343536376B
:1039C000383961626364656678700030313233344F
:1039D0003536373839414243444546585000000097
:1039E00002400000000000A00000000005400000B0
:1039F000000000C8000000000C4000000000409CD7
:103A000000000000194000000020BCBE00000000C3
:103A100034400000BFC91B8E00000004B540000008
:103A2000504BCFD06607E2CF010000006C41000090
:103A30003E8251AADFEEA73401000000D942000007
:103A4000DCB5A0E23A301F97FFFFFFFFB44500004E
:103A5000FD25A0C8E9A3C14FFFFFFFFFFF3F000006
:103A60000000008000000000FF3F00000000008018
:103A7000000000000D0A2A2A2A2A2A2A2A2A2A2A8B
:103A80002A2A2A2A2A2A2A2A2A2A2A2A2A2A2A2A96
:103A90002A2A2A2A2A2A2A2A2A2A2A2A2A2A2A2A86
:103AA0002A2A2A2A2A2A2A2A2A2A2A2A2A2A2A2A76
:103AB0002A2A2A2A000000000D0AB0E6C8A8B9E99F
:103AC000CAF4203A20EACCB3CFBFC6BCBC20323007
:103AD00031372F382D323032372F38202E0909094F
:103AE0000909090D0ABCBCCAF5D6A7B3D6203A20ED
:103AF0004D722E2057616E672020313336333535B5
:103B00003133363138202E00543C020800000020AA
:103B1000980100006CC101081C3D020898010020BA
:103B200028CA0000C8C101081001000043000000BD
:103B3000F8FFFFFF004040404040404040404141CE
:103B40004141414040404040404040404040404072
:103B5000404040404005020202020202020202020C
:103B60000202020202202020202020202020200209
:103B70000202020202029090909090901010101099
:103B80001010101010101010101010101010101035
:103B900002020202020288888888888808080808C9
:103BA0000808080808080808080808080808080895
:103BB00002020202400000000000000000000000BD
:103BC00000000000000000000000000000000000F5
:103BD00000000000000000000000000000000000E5
:103BE00000000000000000000000000000000000D5
:103BF00000000000000000000000000000000000C5
:103C000000000000000000000000000000000000B4
:103C100000000000000000000000000000000000A4
:103C20000000000000000000000000000000000094
:103C300000000000000000001C0000004300000025
:103C4000F8FFFFFF0C0000000E0000000F00000056
:103C50002E00000001142230400E3132312E352E5C
:103C60003231372E323532100F581B7017C9F6011A
:103C700008A1F70108400B3220146840371A2009C8
:103C8000E268280901020209020A0A0C0A17030A5B
:103C9000030B0B0214380140124412401A48041A54
:103CA0004C0412501B4004141A04141A04141A046D
:103CB0001412391C020845041A51041A5D044112F9
:103CC000081C02401C041A30041A44041A58041A2E
:103CD0006C041A80041B08041C19041A30041A44CA
:103CE000041A5804111A08681A0C041A10041A1439
:103CF000041A18041A1C041A200401133C020406B6
:103D00006819A82A040415060708098CA24A04CADF
:0C3D10005914011B1AAA01015400000004
:040000050801C351DA
:00000001FF
